:020000040800F2
:100000000020001001710008E5490008111E0008D9
:10001000E1490008DD490008D94900080000000056
:10002000000000000000000000000000D5490008AA
:10003000D149000800000000CD490008A9230008AC
:100040006971000869710008697100086971000828
:100050006971000869710008C1300008ED310008BD
:10006000B13100087531000839310008595F0008C6
:10007000495F0008395F0008295F0008195F000820
:10008000055F0008F15E00086971000869710008E9
:10009000094B00086971000869710008FD3000080B
:1000A000C920000815210008697100083D210008D9
:1000B00009210008F9200008697100086971000829
:1000C00069710008697100086971000869710008A8
:1000D000697100085924000869710008DD230008CF
:1000E00085300008697100085566000869710008CC
:1000F000D920000869710008E9200008697100082A
:10010000000000000000000000000000697100080D
:100110006971000869710008697100086971000857
:10012000DD5E0008C95E0008B55E0008A15E00083B
:100130008D5E0008697100080000000000000000EA
:100140006971000869710008697100080000000009
:10015000000000000000000000000000000000009F
:1001600000000000000000006971000869710008CB
:10017000697100080000000000000000000000009D
:08018000000000006971000895
:100188002DE9F04FB54E9DB006F1010906F1020BBD
:10019800741E002554F80B0C88B3B14BCC2707FB11
:1001A800053708E0242838D0AE4B9B7E834200F008
:1001B800D28054F80B0C03685B689847F8B154F880
:1001C8000B0C0368DB68984714F8033C002BE9D054
:1001D800012B26D0022B2AD0032B3BD0042B00F076
:1001E800A980052B43D0062BE3D114F8027C002FFD
:1001F8004ED0012F00F0EC80002304F8033C0135B9
:10020800032D06F1CC0609F1CC090BF1CC0B04F156
:10021800CC04BFD11DB0BDE8F08F012304F8033C26
:10022800C7E74D2812D0002304F8033CC1E7002398
:100238003C2804F8033C00F088803E28B9D101220C
:10024800032304F8022C04F8033CB2E7022304F861
:10025800033CAEE7C028E6D80022042304F8060CC5
:1002680004F8050C04F8072C04F8033CA1E714F87B
:10027800073C14F8062C9A4274D814F8053C8342BB
:10028800D1D114F8027C062304F8033C002FB0D126
:10029800754B14F804AC14F806ECADF82A700FCBC3
:1002A8000DF1100888E80F00631E03EB0E010FFA2A
:1002B8008AF20893BAF1380F4FF001030991ADF8AB
:1002C8002820ADF818208DF82C3000F0DF8354D9A1
:1002D800BAF1800F00F0F18300F2A280BAF1520F58
:1002E80000F0BB8440F2DD81BAF1540F00F0F583D1
:1002F800BAF16E0F40F06A825C4ADFF898A1128862
:10030800DAF808100093FF2A594B5A480490A8BFFE
:10031800FF2281F3100189B240461A7006F016FDDB
:100328003946404606F012FDDAF8001001F30F01D5
:1003380089B245E014F8053C04F8040C584005233C
:1003480004F8050C04F8033C33E7032204F8023CE4
:1003580004F8032C2DE7484A484B49491160494A9B
:10036800DA6026E714F8052CF9184240013304F83E
:10037800052C04F8073C88721BE7BAF1040F00F05B
:10038800C18340F28B80BAF1200F00F0458440F21F
:100398006F81BAF1240F00F03384BAF1280F40F0CE
:1003A80015820093DFF8F0A0314B3748374ABAF886
:1003B800001004901A60404606F0C8FCBAF8021013
:1003C800404606F0C3FC0DF1300A009B049A79E020
:1003D80014F8042C14F8063C611E0B4408916E2A8C
:1003E8004FF000010A9109930B91ADF8282000F015
:1003F8003F83B62A7FF400AF14F8012C0894042A2E
:100408003FF6FAAE01A151F822F000BF89070008B3
:10041800010200086707000825070008810700088F
:10042800BAF1820F00F0BA83C0F04F81BAF1A00F81
:1004380000F07B83BAF1FE0F40F0C881144F07F13A
:10044800080A37F8021B404606F080FCBA45F8D186
:10045800049A012300270DF1300A33E0CC0900206B
:10046800C0090020F8140020348800084416002031
:10047800901C0020911C0020FC9F002000ED00E053
:10048800EFBEADDE0400FA05941C002001060A0147
:100498004C160020D01500200C160020BAF1020FCF
:1004A80000F0088100F225839A4540F08F81BA4B0D
:1004B800B94983F801A025221F708A705346CA1CC7
:1004C8000DF1300A54F80B0CADF81A30016805929A
:1004D800D1F820C0B0490491BCF1000F00F091821E
:1004E800E047BDF91A30059A049954F80B0CA2EBB1
:1004F80001080022CAF80020CAF804204246FF2A50
:100508004FF0240E4FF04D01A8BFFF2201338DF8A4
:1005180030E08DF8311000F0A9829DF81C30002BD6
:1005280014BF3C213E21BDF818308DF83210B8F1C7
:10053800FE0F8DF833208DF8343040F364824FEA93
:1005480028238DF8363003238DF835800093072251
:10055800514602F0E9F8009A9DF834309DF83310BE
:100568000132022A83EA01030AD0042A9DF83510D1
:1005780008BF9DF8362083EA010304BF5340DBB26D
:10058800B8F1000F8DF80F3057DD4246049954F842
:100598000B0C02F0C9F8A8F10401890808F1FF3230
:1005A800013104989DF80F300090062A4FEA810A1D
:1005B80040F36A824FF0000E8446CDF804B07046CE
:1005C8005CF804BB0EF1010E71458BEA0000F7D808
:1005D800C0F3072141404B40C0F307414B4000990D
:1005E800DDF804B083EA1063D0455144A2EB0A0257
:1005F800DBB220D00878002A83EA00031BDD4878A4
:10060800012A83EA0003DBB215DD8878022A83EA2F
:10061800000310DDC878032A83EA00030BDD08799C
:10062800042A83EA000306DD4879052A83EA0003E1
:1006380001DD8A7953408DF80F3054F80B0C0122F4
:100648000DF10F0102F070F854F80B0C03685B6AA7
:1006580003B19847002304F8033C002F3FF4CFADC3
:1006680054F80B0C04F010F954F80B0CB847C6E515
:10067800BAF1050F40F0AA800B2248490093404682
:1006880006F042FB08224649404606F03DFB072299
:100698004046444906F038FB0DF1300A009B049AA5
:1006A80010E7BAF1440F40F09180049A3E4F0DF1E3
:1006B800300A07E7042240463C4900930DF1300A0E
:1006C80006F022FB009B049AFCE6394A0193116864
:1006D800314B3848926804904FF6FF7A5145A8BFCD
:1006E80051464FF00A0E21EAE17183F800E089B221
:1006F8004046009206F02AFB009A02EB820149006C
:100708005145A8BF514621EAE17189B2404606F039
:100718001DFB0DF1300A019B049AD3E6A3EB0B03F2
:100728001E2BA8BF1E230DF1300A1A465946504603
:100738006778009394F80080CDF820B007F0CEFFDA
:10074800009B1D481CAA02EB030E3946534600279E
:10075800424600680EF8407C02F084FD4CE5164BDA
:100768001F683B6838469B689847144A0123FF2155
:1007780079733B7313703FE5114B01221A703BE507
:1007880001F0C2FD0F4A104B00F5742000F51070FF
:10079800106000221A702FE5901C0020AC8B000816
:1007A800B88B0008C48B0008B9400008A48B000867
:1007B80010160020911C00204C0C0020520C002028
:1007C800500C00205C0E0020510C0020BAF1650F7F
:1007D80000F01D81BAF1960F00F01981AAF1210AE3
:1007E800BAF1360F00F20881DFE81AF05700060167
:1007F800060106010601060106010601440006017C
:1008080006010601060106010601060106010601A8
:100818000601060106010601060106013700060168
:100828000601060106010601060106010601060188
:100838000601060106010601060106010601060178
:100848000601060106010601060106010601060168
:10085800A80006019A000601730014F8013C0A2B4F
:1008680000F0BE82CDF820B001230DF1300A049AC1
:10087800002727E614F8013C08940A2B08A840F042
:10088800BC8206F035FAB34F388008A806F030FA73
:100898000DF1300A78800123E9E71CA8AE4F14F85F
:1008A800011C2278637840F8509D79703A70BB70CB
:1008B80006F01EFA089B3881591C1A46089112F84E
:1008C800021B797108925B78BB710DF1300A012324
:1008D800CDE704F136030DF1300A14F8012C00922B
:1008E8000893D446274604F1300838687968BA680E
:1008F800FB68E646AEE80F0010374745F446F4D1EA
:100908003868BB88954ACEF80000AEF804301378F2
:10091800002BFCD1924B1F78002F00F01182FEE7CC
:1009280014F8013C0894FF2B66D18E4B2278089668
:1009380083F8702201230DF1300A98E714F8012C8E
:100948000894032A58D8531E87488849DBB203EB1A
:10095800430300EB43030A705878002AEAD00EF1EB
:10096800FF33DBB2834247D10022C1F80220C1F82D
:1009780006208A72002B35D022780896012B8A70BF
:1009880030D06278CDF82090022BCA702AD0A27895
:10099800CDF820B0032B0A7124D0201DE2780890EE
:1009A800042B4A711ED0601D22790890052B8A718C
:1009B80018D0A01D62790890062BCA7112D0E01DCC
:1009C800A2790890072B0A720CD0082BE2794A7298
:1009D80004F108001CBF04F10902237A08901CBF27
:1009E8008B720892624B1B78002BA3D002F0D2FEC8
:1009F8000DF1300A01233AE74FF0FF330DF1300AC9
:100A080035E75C4973E5012300930522A0E55A4BBD
:100A18004046B3F8201106F099F9524BB3F8741216
:100A2800404689B206F092F90021404606F08EF958
:100A38000021404606F072F9049B504A591C0027D1
:100A480004911F7011886429A8BF6421404606F0EC
:100A58007DF9BAF1960F00F065814046394606F0F7
:100A680075F90DF1300A049A01232BE521215AE585
:100A780008A8089406F03CF908A806F039F908A86F
:100A880006F036F9FFF7B8BB0146B3E53C4A3949E9
:100A980092F801E090780B701178364A117182F85B
:100AA80005E005214FF00A0ED7709071517082F859
:100AB80002E00DF1300A073204E53249324A09886A
:100AC800901EFF29A8BFFF214FF00A0E02F8011C53
:100AD80080F800E00DF1300AF4E42B4A2149901E19
:100AE80091F8701202F8011C122101700DF1300A00
:100AF800E8E4204903220A704A708F708A180DF1C1
:100B0800300ADFE4524621490093404606F0FCF8DB
:100B18003946404606F01AF9049A009B511C049184
:100B28001370049A0DF1300ACCE4194A0093116845
:100B3800404606F0F3F8174A4046116806F0EEF80A
:100B4800154A4046116806F0E9F80DF1300A009B95
:100B5800049AB7E40C160020E0150020530C00207E
:100B6800600E0020C00900207C8A000800120020C6
:100B7800DD1A0020901C0020E001002084160020CF
:100B88007C16002054160020921C0020260C002001
:100B9800ACF7FF1FB0F7FF1FB4F7FF1FA549A64A20
:100BA80008781189A54A009302F8010C404604927E
:100BB80006F0CCF8A24A04991288DFF8B4A2FF2AFA
:100BC800A8BFFF22481C04900A70DAF8082082F3B4
:100BD800100291B2404606F0B9F8DAF8001001F3B5
:100BE8000F0189B2404606F0B1F89649049A09788F
:100BF800501C04901170009B049A0DF1300A61E4B6
:100C0800914A0093D2F86C12404606F087F80DF12D
:100C1800300A009B049A55E48C4ADFF81CA2009322
:100C2800D31E9AF801009AF800109AF802E002F828
:100C3800030C59704046BAF8081083F802E0049291
:100C480006F084F8049A9AF80510501C0490117064
:100C5800049A9AF80610501CCBE77D497D4ADFF8C4
:100C680014C20878C2F800C04FF0090E4FF0030C08
:100C780082F805C09371D07182F804E002F1080C83
:100C8800002800F0A7800138C0B2DFF8ECE100EBE3
:100C980040000EEB40004078002800F09B8091F85F
:100CA80002E082F808E001280CF1010240F2B0806D
:100CB800093ACB785372022800F0B5800B79937209
:100CC800032802F10B0300F0A780A3F10B074A7970
:100CD800FA72042803F1010200F098808A793A73C5
:100CE800052803F1020200F09180CA797A73062878
:100CF80003F1030200F08A800A7ABA73072803F125
:100D0800040200F083804A7AFA73082803F1050286
:100D18007CD08A7A3A740DF1300A9A1D0027012393
:100D2800FFF7D0BB049A0123D11804911370049AD9
:100D3800D11804911770049A0DF1300AFFF7C2BB5D
:100D4800454B1868454B4FF0010883F8008002F0C6
:100D580067F9434A384682F8008005F02FFE384686
:100D680005F02CFE092005F029FE009805F026FE66
:100D7800D046A8EB0A07FFB20A2005F01FFE384646
:100D880005F01CFE18F8017B0B2005F017FE38460D
:100D980005F014FE334B186802F038F90DF16603BC
:100DA8004345E6D1082005F009FEA02005F006FE1F
:100DB800A02005F003FE002005F000FE10F0200042
:100DC800F6D1254B0746186802F030F9234B1F70FF
:100DD80001234CE5624607460DF1300AFFF772BB66
:100DE800214B22781A706178A27859709A70CDF8E0
:100DF80020B001230DF1300A39E505F079FF08A884
:100E080005F076FF0DF1300A012330E501230027B4
:100E18000DF1300AFFF756BB1A46002701230DF1E2
:100E2800300AFFF74FBB114A012300270DF1300AA2
:100E3800FFF748BBCC150020E0150020911C0020CE
:100E480044160020881C0020C0090020931C0020A4
:100E580000120020901C002090160020600E002038
:100E68008C160020701B00207C1600209A1C002085
:100E7800D0150020030106027C8A000808B51F4B24
:100E8800002832D01E481A6800210180137813F018
:100E98007F0316D0012B27D0022B24D1527902F0E0
:100EA8000F039B0003F1804303F5B84312061B6848
:100EB8001FD403F44053B3F5805F0ED101230370B0
:100EC8000BE0527A930654BF0378022351064CBFB5
:100ED80043F0010323F0010303700A4B1B681B69ED
:100EE8009847074808BD084608BD1B6802221A82B1
:100EF80008BD03F03003102BEFD1DFE77815002091
:100F0800480C00209C15002008B538B1064B1B681A
:100F18009B689847054B18680C3008BD034B1B6845
:100F280001221A8208BD00BF9C15002078150020F8
:100F380008B538B1064B1B681B689847054B1868FD
:100F48000A3008BD034B1B6801221A8208BD00BF86
:100F58009C1500207815002010B5094C60680368BE
:100F6800DB69984750B9237A0BB9637A33B1606863
:100F78000368DB68984700232372A37210BD00BF83
:100F8800480C00204FF0FF30704700BF002070472A
:100F9800014BD87A704700BF480C002010B40548B0
:100FA8001E2404FB0211014400200B735DF8044B5E
:100FB800704700BF480C002010B50D4C637A83B908
:100FC800D4F81432C01A00280BDD0122094B6272D2
:100FD80060680C22082102F045F9606803685B6AC2
:100FE8009847A07A10B9207A00B9607A10BD00BF7E
:100FF800480C0020D08B000838B50B4C94F81832F8
:1010080005460BB904F010FE084B94F81D121A7827
:1010180094F81C3212F0400F14BF10220D220A441B
:101028001E332A726B7238BD480C00200000002065
:101038000F4B104A1B689BB223F0070303EBC00059
:1010480002443E294FEA42020AD94B09C80604BFA6
:1010580003F1FF339BB29B0243F4004313607047D4
:101068004B08C90748BF01339B021360704700BF94
:10107800505C004006300020054B064A1B689BB2B6
:1010880023F0070303EBC0000244520011607047CD
:10109800505C004002300020704700BF10B50C4B78
:1010A800002093F82C10FFF7C3FF0A4B1B68187A2F
:1010B800082806D10849094B4FF4805410220C80A7
:1010C8001A80A0F10900B0FA80F0400910BD00BFF5
:1010D80084010020781500205C1B00205E1B002086
:1010E8002DE9F041324E3768398A29B93D7A042D05
:1010F80044D0BC8A042504E0BC8AA1428CBF0225E6
:1011080004258C4228BF0C461FFA84F8BB69404668
:101118009847284B1B689BB223F0070303F1005341
:1011280003F540535B00611C1C68A4B204F1005431
:1011380004F5405449104FEA440418BF002306D070
:1011480030F8022B24F8232001338B42F8D1414692
:101158000020FFF791FF7B8A3A8A17481749A2EBCC
:101168000802984430243A824FF44053A7F812807A
:10117800376804800B803D72BDE8F081104B1A7807
:10118800012A06D00C4B072510223D721A80BDE8B3
:10119800F08108480B4A0068074C80B220F007002D
:1011A800024452003020116019702080E3E700BF2C
:1011B80078150020505C00405E1B00205C1B00205E
:1011C800601B002002300020084BDA68D1070BD4DE
:1011D800DA68D20601D502207047DB6813F0040FE5
:1011E80014BF0320042070470120704700200240EC
:1011F80000230360436083608381036143618361EB
:10120800C361036243628362704700BFF0B48B68B6
:101218000F6A0E694D698A69CC693B4333432B4396
:101228004E6A8D6A8F89134302682343334322F43D
:10123800FF422B4322F070020C6813434A68036094
:1012480047608460C260F0BC704700BF02683B49D9
:101258004FF6FE731A4088424FF0000302600360A5
:1012680043608360C36027D0354B98422AD0354B02
:1012780098422DD0344B984230D0344B984239D0D4
:10128800334B98423CD0334B98420FD0324B984264
:101298003CD0324B98423FD0314B984242D0314BF0
:1012A800984245D0304B98421ED070472F4A536819
:1012B80043F07063536070472C4A536843F00F0340
:1012C80053607047294A536843F0F00353607047EE
:1012D800264A536843F4706353607047234A53683F
:1012E80043F4704353607047214A536843F47023B2
:1012F8005360DAE71D4A536843F47023536070471C
:101308001A4A536843F4700353607047184A536885
:1013180043F00F0353607047154A536843F0F003D6
:1013280053607047124A536843F4706353607047C0
:101338000F4A536843F470435360704708000240F3
:101348001C000240300002404400024058000240A5
:101358006C00024080000240080402401C04024065
:101368003004024044040240580402400000024095
:101378000004024000222DE9F04313460F680126BD
:101388004FF0030E04E00133102B02F1020224D0C7
:1013980006FA03F434EA0705F5D10D7905F1FF3CA7
:1013A800BCF1010F0EFA02FC19D96FEA0C0C0468A3
:1013B80004EA0C0404600468954025430560C56888
:1013C800CC790EFA02FC944025EA0C0501332C4333
:1013D800102BC46002F10202DAD1BDE8F083D0F824
:1013E80008800EFA02FC6FEA0C0C08EA0C08C0F838
:1013F800088091F80580D0F8089008FA02F848EAC1
:101408000908C0F80880B0F804801FFA88F828EAAC
:10141800040484808C79B0F804809C4044EA080471
:10142800A4B28480C3E700BFF0B5524D524CAB69FB
:1014380043F0010383B0AB61112104F5217001F081
:1014480029FC04F5217001F0EBFD05F013FA04F511
:10145800217001F0EBFD6B6943F400336B610222EC
:1014680000234FF4C056032569464FF0904000967C
:101478008DF805508DF804208DF806308DF807306A
:10148800FFF778FF4FF0904394F8C823596A3B4818
:101498003B4D3C4E21F470415962596A41F4604118
:1014A8005962596A21F470215962596A41F46021DC
:1014B80059624FF4802303602B68334923F4802357
:1014C8002B60356802F180431222C4F8C42303F567
:1014D8008233012225F48025082784F8C9733560F2
:1014E80084F8CA231D6845F480251D60D4F8C433E8
:1014F8000C3823F01F0603F01F03355802FA03F3D4
:1015080025EA03033350D4F8C43323F01F0603F04D
:101518001F03755802FA03F325EA0303735094F87E
:10152800C933102B0FD0D4F8C41303F1804321F032
:101538001F0003F5823301F01F01C4588A4022437B
:10154800C25003B0F0BDD4F8C43323F01F0503F034
:101558001F032E5802FA03F333432B50D4F8C43335
:1015680023F01F0003F01F0344589A4022434250BF
:1015780003B0F0BD00100240480C002014040140E4
:1015880000040140040401400C040140B64B5968B2
:1015980001F00C0104292DE9F04100F08D810829A2
:1015A80000F07681B14A026001B10021DFF8B8E2AB
:1015B800AF4CDEF80430C3F3031323441E79F6B2AC
:1015C80022FA06F34360DEF80450C5F302252544E9
:1015D8002F7923FA07F78760DEF80450C5F3C22590
:1015E80025442D79EDB2EB40C360DEF82CC04FEAFC
:1015F8001C1C0CF00F0E04EB4E0E1CF0100FBEF866
:1016080014E01FFA8EFE03D0BEF1000F40F0A88050
:101618009646DFF854C2C0F810E0DCF82CE04FEA38
:101628005E2E0EF00F0C04EB4C041EF0100FA48A73
:10163800A4B202D0002C40F090801446DFF828E2D3
:101648004461DEF830C0894C1CF0100F0CBFA44672
:101658009446C0F818C0DEF830C01CF0200F0CBF4C
:10166800A4469446C0F81CC0DEF830C01CF0400FF9
:1016780018BF14460462DEF83040E40502D59142F2
:1016880000F0CC80784C4362D4F830E01EF4805FE0
:1016980057D0914200F02B818362246BA40540F15E
:1016A800CF80714CC362D4F830E04364246B2405C6
:1016B80040F1E0806C49096B83646B490C6BA507AA
:1016C80052D00B6B03F00303012B00F007810B6B67
:1016D80003F00303022B00F036810B6B03F00303C6
:1016E800032B40D0604B196B11F4403F42D1476344
:1016F8005D4B196B11F4402F57D187635A4B196B07
:1017080011F4401F6CD1C763574B196B11F4400F8C
:1017180000F08180196B01F44001B1F5800F00F0F1
:10172800E3801A6B02F44002B2F5000F00F0138157
:101738001B6B03F44003B3F5400F00F0C980BDE80C
:10174800F0818362246BA4057AD59142A9D1AE4277
:10175800A7D14FEA410C6446D5E0B1FBF4F46DE73C
:10176800B1FBFEFE55E7414B03633F4B196B11F488
:10177800403FBCD0196B01F44031B1F5803F00F017
:10178800AF80196B01F44031B1F5003F00F0DF8004
:101798001B6B03F44033B3F5403F04BF334B436343
:1017A800314B196B11F4402FA7D0196B01F440216C
:1017B800B1F5802F00F09680196B01F44021B1F546
:1017C800002F00F0B8801B6B03F44023B3F5402FC3
:1017D80004BF264B8363244B196B11F4401F92D02E
:1017E800196B01F44011B1F5801F75D0196B01F424
:1017F8004011B1F5001F00F0A2801B6B03F44013E9
:10180800B3F5401F04BF194BC363174B196B11F491
:10181800400F7FF47FAF0764BDE8F081AE427FF4EC
:1018280031AF4FEA410CC0F824C0DEF8308018F41C
:10183800805F64465FD18362DEF83040A4058AD4B5
:10184800094CC362246B640501D591423CD0064C17
:101858004364246B24050DD591427FF42BAFAE422F
:101868007FF428AF54005EE00010024000127A00B6
:10187800000000203A4C8364246BA4047FF51CAF5D
:1018880091427FF419AFAE427FF416AF540050E096
:1018980059685A68C1F38341D50301F102010FD594
:1018A800DB6A304A03F00F030133B2FBF3F301FBA9
:1018B80003F101600A4679E62A4A0260002175E6CA
:1018C800294B03FB01F1F4E7AE42C0D14C0022E002
:1018D800244B0364BDE8F081C26315E7026301E7A6
:1018E800426305E7826309E70264BDE8F081AE421E
:1018F8007FF4D2AE4C00DFF868E08462DEF830E0B6
:101908001EF4007F9CD0DFF858E0C462DEF830E0B7
:101918001EF4806F9BD0DFF848E04464DEF830E0C6
:101928001EF4006FA6D00E498464096B8D047FF500
:10193800C3AEC464C1E64FF400438363DEE64FF4EC
:101948000043C363E0E64FF400430363CAE64FF481
:1019580000434363CCE64FF400430364BDE8F081E1
:101968000010024000127A0000093D00F0B504465C
:101978000068D1F808E04B68CF680E6920F00100D4
:101988000D4649692060626822F4405242EA0E021C
:10199800626022683B4322F4B05222F00C023343C7
:1019A80013432360A36823F440730B4395B0A360EB
:1019B8006846FFF7EBFD174B9C4224D0164B9C4220
:1019C80023D0164B9C4222D0154B9C420CBF0F9A39
:1019D800109A23682968180448BF5200B2FBF1F333
:1019E80001FB1322B2EB510F226828BF0133120406
:1019F80005D54FF6F0721A40C3F3420313439BB266
:101A0800A38115B0F0BD0C9AE3E70D9AE1E70E9AB1
:101A1800DFE700BF003801400044004000480040B4
:101A2800004C004038B5084D00242B59CC341846DA
:101A38001BB11B685B68984720B9B4F5197FF4D1CE
:101A4800002038BD012038BDC00900200123122123
:101A5800132241704271037203700371704700BF13
:101A68002DE9F0410B78057BDB43DFB200F113026F
:101A780000F11D0302F8015F9342FBD1DFF890E00B
:101A880000F12701002203F8012F9942FBD114210C
:101A98000524002647FA04F303F00103002B1E4433
:101AA80014BF4FF019084FF00A0814F0010FF6B2EE
:101AB80014BFAC464FF0000C0023CA1810FA82F28B
:101AC8000133434582F814C0F7D15A1E92B201324D
:101AD800013C8B18621C9BB201D01946DAE716F05C
:101AE800010F14BF19240A240022991810FA81F151
:101AF8000132A2420D75F8D113449BB25A1C03441B
:101B0800002192B21975AEF800200261BDE8F0819B
:101B18001C1000202DE9F04FDFF890A0BAF8023031
:101B28000B3383B01FFA83F901F1060B4FF001085C
:101B38004FF0000C002711F801EB3E464C460122FD
:101B4800A4F10B039BB2019105E001339BB2017B29
:101B580029759C4208D0C518002AF6D1C51801334A
:101B68009BB29C422A75F6D103190136092F0199B7
:101B780083F814C0F6B20CD0092E15D008FA07F372
:101B880013EA0E0F14BF012200220C34A4B201374D
:101B9800D6E709F1780959451FFA89F9CAD1AAF88F
:101BA80002C003B0BDE8F08F0022EEE71C10002051
:101BB8002DE9F047DFF85C80B8F8043004331FFAE9
:101BC80083FC01F109094FF0010E11F8017B64460D
:101BD8000026231F0EFA06F29BB23A40C2B1B0F8B3
:101BE8000CA0C51801339BB29C4285F814A0F5D10E
:101BF80001360434082EA4B2EBD10CF1200C49456F
:101C08001FFA8CFCE1D10023A8F80430BDE8F08766
:101C18009246E6E71C10002010B50168047B0A68AC
:101C28000223A3401A420AD0054A406800241470CF
:101C3800026822F001021204120C02604B6010BD0F
:101C4800DF1A0020436A8269D154436A0169826BB2
:101C580001338B4228BF00234362002A2FD0EFF3C1
:101C68001181502383F31288836B1A68D2072CD40E
:101C780070B45E686EB9456A826A954217D0846905
:101C88001444DC600ED9AA1A5A608562002280F8D2
:101C980054201A6842F00102C9B21A6081F311880F
:101CA80070BC70470469A21A5A608662EEE7012385
:101CB80080F85430C9B281F3118870BC7047026D46
:101CC800136843F0800313607047C9B281F3118829
:101CD800704700BF426B10B462B1436CC26844697C
:101CE800D11A013B615C5DF8044B08BF134643649D
:101CF800C8B27047016A4369C4685B5C0131A1429C
:101D080028BF114601625DF8044BD8B2704700BF86
:101D1800836B13B190F854007047836A406A181AAD
:101D2800B0FA80F040097047416A836A99420AD341
:101D3800CB1A816B026961B14968501E0B4483421A
:101D48000AD2C01A704702691144CB1A816B002964
:101D5800F2D1501EC01A7047002070472DE9F04795
:101D68000569C3681D4028D00F4606464FF0004855
:101D78004FF00009B5FA85F328FA03F2D2431B3B6A
:101D880032611540042B16D8DFE803F031292119F8
:101D980003007B6A002B32D003F1FF3A1FFA8AFA5C
:101DA800C7F824903C6A34B12368204651469847C6
:101DB8006468002CF8D1002DDCD1BDE8F0873868C4
:101DC800716B036889B29847002DD3D1F5E778681D
:101DD800B16B036889B29847002DCBD1EDE7B8689D
:101DE800F16B036889B29847002DC3D1E5E7F8681D
:101DF800316C036889B29847002DBBD1DDE7F36ADF
:101E08001FFA83FACEE700BF184C08B5012102205B
:101E180001F01CF9A37903F00903092B08D000216C
:101E2800012001F013F90021084601F00FF9FEE73F
:101E38000F4A104B11681A680B68A0684FF6FE75B8
:101E48002B400B60138823F001031B041B0C138029
:101E580018B12A2200238271C37102224E2100F098
:101E680047FDA06801F0DCF8D9E700BF1C1000208E
:101E7800E81A0020EC1A0020054B10B5DA68054C6A
:101E88002178501C09B9DA6010BD0246F8E700BF96
:101E98001C100020DF1A00202DE9F04FF02200214D
:101EA80083B07848784CDFF80492784D784E794FB3
:101EB800DFF8FC8106F037FC77487849DFF8F4E171
:101EC800DFF8F4C100221359834200F0C180B3F156
:101ED800804F00F0BF80AB4200F0C880B34200F0F2
:101EE800C780BB4200F0C680734500F0C5806345DB
:101EF80000F0C480434500F0C380DFF8C0A153451B
:101F08007ED00AF5806A534508BF092379D0143278
:101F1800F02AD8D15C4C624D624E604F04F1F00853
:101F280002E01434A04568D0A379002BF9D02379B6
:101F38004FEA131909F1FF39B9F1050F03F00F033F
:101F4800EFD835F8190040FA03F2D207E9D54FF077
:101F5800010A0AFA03F3013B184005F0B9F816F82C
:101F680009305149184411EBC002DAD051F8300059
:101F78004E4B217A00F1384E03EB9E2393F85030F4
:101F880003F01F0E5B09022B0AFA0EFA69D0032B25
:101F980062D0012B03D17B694AEA03037B619388F2
:101FA8000093B3FA83F3C3F11F039BB2DA0800EB83
:101FB800820203F00703D2F820E09B004FF00F0CD9
:101FC8000CFA03FC2EEA0C0EC2F820E0D2F820E04E
:101FD80001FA03F343EA0E0313626946002302225F
:101FE80014348DF804208DF805308DF806308DF8FE
:101FF8000730FFF7BFF9A04596D103B0BDE8F08FD1
:10200800082309EBC3034FF0010B93F804A00AF06F
:102018001F034FEA5A1ABAF1020F0BFA03F30BD057
:10202800BAF1030F0ED0DA457FF471AFD1F814A0DE
:1020380043EA0A034B616AE7D1F818A043EA0A03A6
:102048008B6164E7D1F81CA043EA0A03CB615EE721
:102058000023D6E70123D4E7FB694AEA0303FB61BF
:102068009DE7BB694AEA0303BB6198E70223C8E717
:102078000323C6E70423C4E70523C2E70623C0E712
:102088000723BEE72C1000205089000800040040F8
:102098000008004000100040002C014000100240E1
:1020A8004C880008448800086C0E002058880008F6
:1020B8000040014000140040003401400044014049
:1020C800014902484AE600BFCC1000200040014008
:1020D8000149024842E600BFA41000200034014034
:1020E800014902483AE600BFA4100020003401402C
:1020F8000149024832E600BF7C100020000400407D
:1021080001494FF0804029E65410002010B5064CD4
:10211800064804F11001FFF721FE04F1D801044834
:10212800BDE810401AE600BF1C100020002C01403A
:10213800004401400149024810E600BF2C1000206D
:10214800002C01401F4B98422CD0B0F1804F2BD06F
:10215800A3F59433984229D003F58063984227D099
:1021680003F50063984225D003F58063984223D095
:1021780003F59033984221D003F5406398421FD06D
:1021880003F58063984207D003F58063984208BF3F
:10219800092202D00020704708220B4B03EBC20330
:1021A800187970470022F8E70122F6E70222F4E7DF
:1021B8000322F2E70422F0E70522EEE70622ECE725
:1021C8000722EAE7002C0140588800082DE9F04F63
:1021D800DFF830C1474A4849484E494D80461027E4
:1021E80018F1FF38C0F08480DCF80430C3F308032A
:1021F800002B5CD1EFF31183002B58D10B68946846
:1022080000BF08688342F9D1D6F800904FF47A707D
:1022180000FB09FEAEEB040EBEFBF9FE00FB03EE6D
:10222800DCF80430C3F308034FF47A740120FBB9D7
:10223800EFF31183E3B90B68D2F808A000BFD1F817
:1022480000904B45F7D1D6F800B004FB0BF9A9EB89
:102258000A09B9FBFBF904FB0393A3EB0E03B3F5DF
:102268007A7FBDD2DCF80430C3F30803002BDFD03B
:10227800EFF3118A87F31288D2F808B01368DB03EA
:1022880044BF2860D2F808B00B68D5F800905FFA10
:102298008AFA8AF31188D6F800A0994404FB0AF355
:1022A800A3EB0B03B3FBFAF304FB0933D5E7EFF316
:1022B800118487F31288D2F808901368D80303D5DD
:1022C80001232B60D2F808900B682868E4B284F3E5
:1022D8001188D6F800A04FF47A7400EB030E04FBC3
:1022E8000AF3A3EB0903B3FBFAF304FB0E3E97E7EB
:1022F800BDE8F08F10E000E0401C0020441C0020E6
:102308003C1C002000ED00E0204B5B68C3F3080391
:1023180030B4BBB9EFF31183A3B91D4B1D4C18683A
:10232800A16800BF1A689042F9D11B4B1C684FF492
:102338007A7202FB04F3591AB1FBF4F130BC02FBC8
:1023480000107047EFF31182102383F312881149AC
:102358008C680B6813F4803F104B02D00120186082
:102368008C680B49D2B20D68186882F311880A4B41
:1023780019684FF47A72284402FB01F31B1B30BC26
:10238800B3FBF1F302FB0030704700BF00ED00E043
:10239800401C002010E000E0441C00203C1C0020F1
:1023A80030B4EFF31183102282F312880649074CE8
:1023B8000A680748013200250A602560DBB2026816
:1023C80083F3118830BC7047401C00203C1C00205F
:1023D80010E000E01D4B70B59C68236D626BDD69F1
:1023E800C2B1A36B2BB12B0702D5236D08221A6249
:1023F80070BD2A06F7D5A26A616A8A4220D0511CAC
:10240800A069A162825C2069266D81423285EAD387
:10241800A362E8E7A906E4D5E26A22B1988C216BA9
:1024280080B29047DDE7E1699B8C6069DBB24E1CA6
:10243800E6614354E169E368994228BFE261D0E765
:10244800226D136823F080031360CCE7EC110020A1
:102458001D4B70B51C68236D626BDD69C2B1A36B3F
:102468002BB12B0702D5236D08221A6270BD2A06EC
:10247800F7D5A26A616A8A4220D0511CA069A1627C
:10248800825C2069266D81423285EAD3A362E8E73F
:10249800A906E4D5E26A22B1988C216B80B29047F4
:1024A800DDE7E1699B8C6069DBB24E1CE661435451
:1024B800E169E368994228BFE261D0E7226D1368B9
:1024C80023F080031360CCE7EC110020436B43B189
:1024D800426C5B6893422FBF981AC0689B1AC01859
:1024E8007047C269036A9A422FBFD01AC068801821
:1024F800C01A70471A232B228372192303700273A0
:1025080000232A22037582708375704700231F22D7
:10251800027043708370C3707047152303701623CD
:10252800C370172383712D2343702E2303712F2328
:10253800C371704730B50446006D61710368A268C5
:1025480023F00103036087B0A379009213F004021B
:102558003DD04FF4805213F00203019244D102930C
:102568004FF480630022039311F00103059237D1E1
:10257800049308238D07694648BF0493FFF7F6F9CB
:102588006079236DA17900F00202002A15BF4FF48B
:1025980040324FF480324FF40034002410F0010F21
:1025A800586808BF2246CC074CBF024320EA020203
:1025B8005A609A6809074CBF42F0080222F00802E4
:1025C8009A601A6842F001021A6007B030BD13F031
:1025D800020301920BD04FF4005513460295C1E750
:1025E800042304930C23C5E74FF40053B7E7029381
:1025F800B8E700BF10B50446006DA160036823F07A
:1026080001030360A37986B013F00402009141D05E
:102618004FF4805213F00203019244D102934FF415
:10262800806362790393D1074FF000030493059305
:1026380045BF0423049308230C236946920748BF27
:102648000493FFF793F96079236DA17900F00202F2
:10265800002A15BF4FF440324FF480324FF4003453
:10266800002410F0010F586808BF2246CC074CBF61
:10267800024320EA02025A609A6809074CBF42F0F6
:10268800080222F008029A601A6842F001021A60F1
:1026980006B010BD13F00203019207D04FF40051A9
:1026A80013460291BDE74FF40053B7E70293B8E72A
:1026B80000232622036002702722827001224360D1
:1026C80002718371704700BF70B4EFF31186502315
:1026D80083F31288836B1A68D20720D45D686DB9BA
:1026E800446A826A944217D081691144D9600ED92C
:1026F800A21A5A608462002280F854201A6842F0B4
:102708000102F1B21A6081F3118870BC7047016947
:102718008A1A5A608562EEE7012380F85430F1B2D4
:1027280081F3118870BC704703682DE9F041DF69B7
:102738001FB13B46BDE8F0411847002A164611DD97
:1027480004460D460E4400E023689B6820469847DF
:102758000028F9D0236815F8011B1B682046984704
:10276800AE42F1D1BDE8F08110B50409013C052C59
:1027780017D80D4B33F8142000F00F0042FA00F37D
:1027880013F001030DD0012303FA00F001381040C3
:1027980004F09EFC054A064B125D104403EBC00092
:1027A80010BD002010BD00BF4C88000844880008F8
:1027B8006C0E00202DE9F04F4A484B4B4B4C4FF024
:1027C80090414FF0010A4FF002094FF004084FF012
:1027D800080C4FF0100E20274026802530F8022BD9
:1027E80012F0010F03D01960A3F804A0083312F007
:1027F800020F03D01960A3F80490083312F0040FF5
:1028080003D01960A3F80480083312F0080F03D02E
:102818001960A3F804C0083312F0100F03D0196030
:10282800A3F804E0083312F0200F02D019609F804B
:10283800083312F0400F02D019609E80083312F05E
:10284800800F02D019609D80083312F4807F05D074
:102858004FF4807B1960A3F804B0083312F4007FAA
:1028680005D04FF4007B1960A3F804B0083312F4C4
:10287800806F05D04FF4806B1960A3F804B008335B
:1028880012F4006F05D04FF4006B1960A3F804B080
:10289800083312F4805F05D04FF4805B1960A3F809
:1028A80004B0083312F4005F05D04FF4005B1960E0
:1028B800A3F804B0083312F4804F05D04FF4804BCE
:1028C8001960A3F804B00833D20B04D04FF40042C7
:1028D80019609A80083301F58061A1427FF47EAFC8
:1028E800BDE8F08F4C8800086C0E002000180048E6
:1028F800002867D003682DE9F04F03F138445C4E97
:10290800A40A0125345D04F01F066409022C05FAA7
:1029180006F558D0032C00F0A580012C58D08088EB
:10292800B0FA80F4C4F11F04A4B2E50803EB8505EE
:1029380004F007042E6AA4000F27A74026EA07061A
:102948002E622E6A01F00307A2407C1E3243012C3E
:10295800C1F3810CC1F300182A62C1F341113CD9BB
:10296800C60700F18980850700F19580440700F1CA
:10297800A380020700F1B180C60600F1BF8085067A
:1029880000F1CD80440600F1DB80020600F1E98009
:10299800C60500F1F780850500F10581440500F1C1
:1029A8001381020500F12181C60400F12F818504FD
:1029B80000F13D81440400F14B81020400F159818A
:1029C800BDE8F08F70472B4CA6693543A561A6E793
:1029D800284C666935436561A1E7002422464FF01B
:1029E800010E4FF0030904E00132102A04F1020439
:1029F800E6D00EFA02F636EA0005F5D1D3F808A0BB
:102A080009FA04F5ED430AEA050AC3F808A0D3F861
:102A180008B00CFA04FA4AEA0B0AC3F808A0B3F89B
:102A280004A01FFA8AFA2AEA06069E80B3F804A0D0
:102A380008FA02F646EA0A06B6B29E801E682E40DA
:102A48001E60D3F800A007FA04F646EA0A061E60DC
:102A5800D3F80CA001FA04F605EA0A0A46EA0A05C0
:102A6800DD60C1E7034CE6693543E56157E700BF20
:102A7800A8880008001002401A6822F003021A60B1
:102A88001A683A431A60DA6822F003020A43850793
:102A9800DA607FF56BAF1A6822F00C021A601A68C8
:102AA80042EA87021A60DA6822F00C0242EA8102DE
:102AB8004407DA607FF55DAF1A6822F030021A60C9
:102AC8001A6842EA07121A60DA6822F0300242EA0B
:102AD8000112DA6002077FF54FAF1A6822F0C002D0
:102AE8001A601A6842EA87121A60DA6822F0C0028D
:102AF80042EA8112C606DA607FF541AF1A6822F40D
:102B080040721A601A6842EA07221A60DA6822F4E8
:102B1800407242EA01228506DA607FF533AF1A680F
:102B280022F440621A601A6842EA87221A60DA6858
:102B380022F4406242EA81224406DA607FF525AF3A
:102B48001A6822F440521A601A6842EA07321A6078
:102B5800DA6822F4405242EA0132DA6002067FF56E
:102B680017AF1A6822F440421A601A6842EA87329C
:102B78001A60DA6822F4404242EA8132C605DA6015
:102B88007FF509AF1A6822F440321A601A6842EADF
:102B980007421A60DA6822F4403242EA01428505A7
:102BA800DA607FF5FBAE1A6822F440221A601A68D0
:102BB80042EA87421A60DA6822F4402242EA8142F5
:102BC8004405DA607FF5EDAE1A6822F440121A6007
:102BD8001A6842EA07521A60DA6822F4401242EA96
:102BE8000152DA6002057FF5DFAE1A6822F440026E
:102BF8001A601A6842EA87521A60DA6822F44002B8
:102C080042EA8152C604DA607FF5D1AE1A6822F032
:102C180040721A601A6842EA07621A60DA6822F09B
:102C2800407242EA01628504DA607FF5C3AE1A6831
:102C380022F040621A601A6842EA87621A60DA680B
:102C480022F0406242EA81624404DA607FF5B5AE60
:102C58001A6822F040521A601A6842EA07721A602B
:102C6800DA6822F0405242EA0172DA6002047FF523
:102C7800A7AE1A6822F040421A601A6842EA8777BB
:102C88001F60DA6822F0404242EA8171D960BDE8EB
:102C9800F08F00BF002852D0036803F138422DE9B5
:102CA800F04F920A504DAA5C02F01F055209012408
:102CB800022A04FA05F443D0032A00F09080012A7E
:102CC80043D001F003077A1E012AC1F3810CC1F336
:102CD80000188088C1F341113CD9C60700F18880EB
:102CE800850700F19480440700F1A280020700F1F3
:102CF800B080C60600F1BE80850600F1CC8044068F
:102D080000F1DA80020600F1E880C60500F1F680DD
:102D1800850500F10481440500F11281020500F1E6
:102D28002081C60400F12E81850400F13C81440411
:102D380000F14A81020400F15881BDE8F08F704724
:102D48002A4A95692C439461BBE7284A55692C4364
:102D58005461B6E7002422464FF0010E4FF00309F4
:102D680004E00132102A04F10204E6D00EFA02F659
:102D780036EA0005F5D1D3F808A009FA04F5ED43C1
:102D88000AEA050AC3F808A0D3F808B00CFA04FA4E
:102D98004AEA0B0AC3F808A0B3F804A01FFA8AFA93
:102DA8002AEA06069E80B3F804A008FA02F646EA64
:102DB8000A06B6B29E801E682E401E60D3F800A098
:102DC80007FA04F646EA0A061E60D3F80CA001FAD0
:102DD80004F605EA0A0A46EA0A05DD60C1E7034A7D
:102DE800D5692C43D4616CE7A8880008001002401C
:102DF8001A6822F003021A601A683A431A60DA68FD
:102E080022F003020A438507DA607FF56CAF1A687F
:102E180022F00C021A601A6842EA87021A60DA681D
:102E280022F00C0242EA81024407DA607FF55EAFC5
:102E38001A6822F030021A601A6842EA07121A6009
:102E4800DA6822F0300242EA0112DA6002077FF5FE
:102E580050AF1A6822F0C0021A601A6842EA871254
:102E68001A60DA6822F0C00242EA8112C606DA6005
:102E78007FF542AF1A6822F440721A601A6842EA73
:102E880007221A60DA6822F4407242EA01228506B3
:102E9800DA607FF534AF1A6822F440621A601A6863
:102EA80042EA87221A60DA6822F4406242EA812202
:102EB8004406DA607FF526AF1A6822F440521A6099
:102EC8001A6842EA07321A60DA6822F4405242EA83
:102ED8000132DA6002067FF518AF1A6822F4404220
:102EE8001A601A6842EA87321A60DA6822F44042A5
:102EF80042EA8132C605DA607FF50AAF1A6822F421
:102F080040321A601A6842EA07421A60DA6822F404
:102F1800403242EA01428505DA607FF5FCAE1A6864
:102F280022F440221A601A6842EA87421A60DA6874
:102F380022F4402242EA81424405DA607FF5EEAE8F
:102F48001A6822F440121A601A6842EA07521A6094
:102F5800DA6822F4401242EA0152DA6002057FF58B
:102F6800E0AE1A6822F440021A601A6842EA8752F0
:102F78001A60DA6822F4400242EA8152C604DA6032
:102F88007FF5D2AE1A6822F040721A601A6842EAD7
:102F980007621A60DA6822F0407242EA0162850428
:102FA800DA607FF5C4AE1A6822F040621A601A68C7
:102FB80042EA87621A60DA6822F0406242EA816275
:102FC8004404DA607FF5B6AE1A6822F040521A60FF
:102FD8001A6842EA07721A60DA6822F0405242EA36
:102FE8000172DA6002047FF5A8AE1A6822F0404246
:102FF8001A601A6842EA87771F60DA6822F040424E
:1030080042EA8171D960BDE8F08F00BF30B1026833
:103018008388918A0B4218BF1B049361704700BFD5
:1030280010B1036882881A85704700BF10B1036821
:1030380082889A61704700BF38B100298388026886
:1030480014BF002110218B409361704710B4094BC5
:10305800094A1C7801238340234052F8200029B9EB
:10306800B3FA83F149095DF8044BE5E7191C18BF69
:103078000121F8E76C1B0020701B00202DE9F041AE
:103088000B4E346873691C400FD0DFF82880012785
:10309800B4FA84F3C3F11F0307FA03F558F82300C1
:1030A80003689847AC437561F2D1BDE8F08100BF71
:1030B80000040140341100202DE9F0410B4E346822
:1030C80073691C400FD0DFF828800127B4FA84F315
:1030D800C3F11F0307FA03F558F82300036898475C
:1030E800AC437561F2D1BDE8F08100BF0004014036
:1030F800341100202DE9F0410B4E346873691C40EF
:103108000FD0DFF828800127B4FA84F3C3F11F0336
:1031180007FA03F558F8230003689847AC4375612C
:10312800F2D1BDE8F08100BF000401403411002055
:103138002DE9F0410B4E346873691C400FD0DFF85D
:1031480028800127B4FA84F3C3F11F0307FA03F5B3
:1031580058F8230003689847AC437561F2D1BDE87D
:10316800F08100BF00040140341100202DE9F04136
:103178000B4E346873691C400FD0DFF82880012794
:10318800B4FA84F3C3F11F0307FA03F558F82300D0
:1031980003689847AC437561F2D1BDE8F08100BF80
:1031A80000040140341100202DE9F0410B4E346831
:1031B80073691C400FD0DFF828800127B4FA84F324
:1031C800C3F11F0307FA03F558F82300036898476B
:1031D800AC437561F2D1BDE8F08100BF0004014045
:1031E800341100202DE9F0410B4E346873691C40FE
:1031F8000FD0DFF828800127B4FA84F3C3F11F0346
:1032080007FA03F558F8230003689847AC4375613B
:10321800F2D1BDE8F08100BF000401403411002064
:103228000D490E4B8A6942F0010210B58A611A688D
:103238000B4C42F400621A601A6842F480521A6019
:1032480020464022002105F06EFA4FF0FF33236438
:10325800C4F8433010BD00BF001002400000014018
:10326800341100202DE9F041044618460D46164653
:10327800984603F025FF2768E6722844A07229467D
:103288007D69434632462046AC46BDE8F04160477A
:1032980098B10B4B012210B402FA01F103F1750445
:1032A80002E00333A34209D01A788242F9D15A784E
:1032B8000A42F6D001205DF8044B70470020FAE777
:1032C800B088000810B40023094C01E0272B0AD06D
:1032D80003EB43020133A15C8142F7D122445DF83C
:1032E800044B9078704700205DF8044B704700BF8E
:1032F800B0880008F8B504460D468E180027B54278
:1033080001D12069F8BDE368591CE160234415F830
:10331800012B1A720429F2D1A168204603F09FFB01
:10332800E7602061EBE700BFF0B51C78002A0CBF0E
:103338004FF0200E4FF0300E5D1C4CB300292BDDF2
:103348002E4601E01146AAB116F8017B4A1E002F4D
:10335800F8D18E1E72B13146046801394A1C671CC7
:10336800002A076084F800E0F6DC1C7826EAE6719B
:103378004A1C5CB1D21A0368591C01601C70AB1856
:1033880015F8014B002CF6D11846F0BD1346FBE7A3
:10339800002903DC2346F7E70022EBE74E1EDAE7B5
:1033A800F0B40D6800240BE0052B18D8A0F1370302
:1033B8000A2B14DC04EB840415F8010B03EB44041A
:1033C800A0F13003DEB2092EA0F16107F2D9052F72
:1033D800A0F14103E8D8A0F157030A2BEADD0D60FC
:1033E8001460F0BC704700BF2DE9F043544B53F80C
:1033F800204083B0002C00F08880A56D514F4FF419
:10340800807304F5AF7206466868A16004F15E0136
:10341800276020656161A261E3602361287E03F073
:10342800AFFAEF68FFB1DFF828E10023714648687A
:10343800874201F11C0103D001330C2BF7D1002383
:10344800C3EBC3030EEB83033F481A6941694FF08E
:103458000C0E1143721C416183F818E05A76236DF3
:1034680067632433E364AF683FB3DFF8E4E0002226
:1034780071464868874201F11C015ED001320C2A6E
:10348800F7D100221046C2EBC2020EEB8202DFF82F
:10349800B8E01769DEF814302C493B43CEF81430F5
:1034A8000B27731C53761776EA7E234602F0C6FC78
:1034B800236DAA68A2632833A36494F85D00FFF71C
:1034C80053F9074694F85C00FFF74EF995F8199000
:1034D800804647B10B22731CBA71FB7138464A46C5
:1034E8002E21FFF705FAB8F1000F0AD001360C2398
:1034F80088F807604A4688F8063040462E21FFF7CC
:10350800F7F9636B2BB1A36B1BB1204603B0BDE881
:10351800F0832B7FAA7E8DF804209B0900210122CD
:1035280001A88DF805308DF806108DF8072003F0F6
:103538006FFA204603B0BDE8F083D0B2A3E700BF1E
:10354800EC11002028890008001002400D5C0008DA
:1035580034000020DFED827A20EE270AFDEEC07AE3
:1035680017EE903A2033402B00F28C80DFED7D7A05
:10357800B4EEE70AF1EE10FA40F3E880B0EE407AD4
:103588009FED796ADFED796A01E0B0EE677AB4EE13
:10359800E67AF1EE10FA77EE467AF6DC9FED747A69
:1035A800F4EEC77AF1EE10FA40F1CD809FED6E6A25
:1035B800DFED706A01E0F0EE477AF4EEE67AF1EEBC
:1035C80010FA37EE867AF6D4DFED6B7AB4EEE77A46
:1035D800F1EE10FA51DCDFED697AB4EEE77AF1EE3C
:1035E80010FA44BFDFED627A37EEC77A27EE076A32
:1035F800DFED635ADFED637ADFED636A9FED635AAF
:10360800E6EE257A67EE065AE6EE276AF7EE007AC6
:10361800A5EEA67AF0EE675AE7EE055AE7EE457A88
:1036280087EEA55ADFED547A30EE277AFDEEC76AA9
:1036380016EE903A2033402B29D99FED557AF6EEB5
:10364800006AB7EE006AF7EE004AC4EEA57A0023D6
:10365800836143610362C36180ED045A67EEA66A21
:1036680027EE866A27EE877AC0ED006AC0ED026A07
:1036780080ED016A80ED037A7047DFED3A7A37EE24
:10368800C77AB3E7B7EE005AF0EE455ACAE7B4EE88
:10369800E70AF1EE10FA5FDD9FED336ADFED336A7A
:1036A80001E0B0EE677AB4EEE67AF1EE10FA77EE62
:1036B800467AF6DC9FED2E7AF4EEC77AF1EE10FA30
:1036C80047D59FED296ADFED2B6A01E0F0EE477AD6
:1036D800F4EEE67AF1EE10FA37EE867AF6D4DFEDFC
:1036E800267AB4EEE77AF1EE10FA27DCDFED237ADA
:1036F800B4EEE77AF1EE10FA44BFDFED1D7A37EE4B
:10370800C77A27EE076ADFED1E4ADFED1E6ADFED96
:103718001E7AE6EE246A67EE064AE6EE267AB7EEE9
:10372800006AA4EEA77AF6EE006A36EE476AF8EE6B
:10373800007A27EE277A66EE266A84E7DFED097AB3
:1037480037EEC77ADDE7B0EE677A3DE7F0EE407A0C
:1037580024E7B0EE677AC2E7F0EE477AAAE700BF3F
:103768007CD9A03EDB0F4940DB0FC940E4CB1641B2
:10377800DB0F49C0E4CB16C1DB0FC93FDB0FC9BF64
:1037880092E741B99730083C15A82ABEF304353FA3
:103798000000008010B5FEF76FFB0548D0F8043331
:1037A80000F116011B682030BDE81040184700BF23
:1037B800EC11002050B1202809D021280ED024284F
:1037C8000ED025280ED018280ED0002070470023D0
:1037D800064803EB830300EB830070470123F7E7F8
:1037E8000223F5E70323F3E70423F1E750890008F0
:1037F8000EB42DE9F04189B010AD684B019000245A
:103808000295039326465622019B591C01910134C7
:103818001A70039B5A1C03921A78002A3ED0252A54
:10382800F2D19A1C049603925878302858D0002771
:10383800A0F13003DBB2092B39D96C283DD06428BC
:1038480000F096800FD8252847D06CD9582878D012
:103858006328DED1019B2A78591C01911A70013422
:103868000435039BD6E7732853D05FD9752865D1F3
:103878000DF114082868434600220A21043503F094
:10388800A1F943463A46049901A8FFF74DFD039B69
:103898005A1C03921A780444002AC0D1019B0022C2
:1038A80020461A7009B0BDE8F04103B0704704AA79
:1038B80003A9FFF775FD6C28C1D1039B1A46013394
:1038C80003931278642A5BD00FD8252A05D05FD9D4
:1038D800582A11D0632ABDD09CE7019B252294E782
:1038E800DA1C039298780127A2E7732A11D052D9DB
:1038F800752A33D0782A8DD1A2F158014A420DF1A8
:1039080014084A41286843461021043503F05AF93F
:10391800B7E72B680499002201A8FFF705FD0435D5
:103928000444039B76E70028B8D072E76E287FF43A
:1039380070AF039B2A68043514606BE778287FF41E
:1039480068AFA0F158035A420DF114085A4128688B
:103958004346102103F036F9043592E70DF11408B7
:103968002868434600220A21043503F02BF988E72A
:103978000DF1140828684146043503F0F5F880E78E
:103988000DF1140828684146043503F0EDF878E78E
:10399800002A83D03EE76E2ACCD03BE79D8B0008F7
:1039A8001E4A92F80833022B33D802EBC30118469B
:1039B800B1F80C130133C907DBB224D4032B28D088
:1039C80002EBC30110B4B1F80C430230E407C1B2F2
:1039D80018460CD4022903D1B2F81C33DB070FD4E4
:1039E800032382F8083300205DF8044B70470B4628
:1039F8000B4982F8083301EBC0005DF8044B7047AF
:103A080008460323F4E7064982F8083301EBC000AF
:103A1800704782F808330020704700BFEC1100207F
:103A2800F81400202DE9F0418C4E96F97A33834240
:103A38008CB00DD096F98233834200F0FE8096F95F
:103A48008A33834200F0FB8000200CB0BDE8F0818F
:103A58000027FF00F319B3F87843002CF4D10228AB
:103A68008846054607D0142800F0C48018B12046BF
:103A78000CB0BDE8F081EDB228464146FFF7B4FC32
:103A880004460028F3D0006D00230322A37162715D
:103A98000268236222F001020121E361A3626362EA
:103AA800E362236384F85410C4F8088001A9026013
:103AB8000C2202930393049306930592CDF8048095
:103AC800FDF754FF6079236DA17900F00202002A06
:103AD80015BF4FF440324FF480324FF4003E4FF0A0
:103AE800000E10F0010F586808BF724611F0010F60
:103AF80014BF024320EA02025A609A6809074CBFC1
:103B080042F0080222F008029A601A68616B42F0DB
:103B180001021A60002900F0998001A8FDF768FBEE
:103B2800E36CE2686169606B01934FF480530A9318
:103B3800002302910B938021059307930893039325
:103B48002023ADF8102009930691FDF77FFB01A90A
:103B5800606BFDF75BFB626B236D116841F001013F
:103B68001160996841F040019960526892B26264AC
:103B7800A26B002A65D001A8FDF73AFBA26C236965
:103B880001924FF480524FF00008A06B0A92ADF8F2
:103B980010308022102306920393CDF82C80CDF8A4
:103BA8001480CDF81C80CDF82080CDF82480FDF756
:103BB8004DFB01A9A06BFDF729FBA26B236D1168D2
:103BC80041F002011160C2F80480C2F804809A68CA
:103BD80042F080029A601A6842F0010220461A6098
:103BE8003E4401230571C6F87403A6F878330CB077
:103BF800BDE8F081FDF718FC194B1A491C60CA6929
:103C0800194B1A4CC6F88C4342F40002CA6103F5FA
:103C1800A87003F5C0710222C6F8AC03D3F850317E
:103C2800C6F8B01386F89823984700F027FF104B82
:103C3800C6F82833A4F16800D2E7012709E702276C
:103C480007E71A6842F080021A60C4E720221A6265
:103C58001A6842F020021A608AE700BFEC110020BF
:103C6800D800424200100240340000207C15002099
:103C7800408A0008104BB3F80C23D1074FF000001E
:103C88000CD4B3F81423D20710D4B3F81C0310F0E3
:103C980001000ED1032283F8082370470246012150
:103CA800064883F8081300EBC2007047022101227E
:103CB800F6E703210222F3E7EC110020F8140020B4
:103CC80030B40D4A0023142502240320C2F87833A7
:103CD800C2F88033C2F88833C2F87C33C2F8843320
:103CE800C2F8743382F8823382F87A5382F88A43AE
:103CF80082F8B40330BC7047EC1100204448454AB0
:103D0800B0F80C134B0830B403F077338D08CB1A96
:103D180005F03335CC0804F011345B1B1B1B03EB97
:103D2800231303F00F3382FB03421A44D211C2EB70
:103D380002229A1A012A01F0010405DD022A65D13E
:103D480001F08101812961D1B0F814536908EA07AB
:103D580001F077314FEA9502A5EB010102F0333209
:103D68004FEAD503A1EB020203F01133A2EB0303E0
:103D780003EB2313274A03F00F3382FB03121A4481
:103D88004FEAE212C2EB022248BF0134A3EB02025F
:103D980048BFE4B2012A05DD022A37D105F08105C2
:103DA800812D33D1B0F81C53690801F07731AA0886
:103DB800EB07A5EB010102F033324FEAD503A1EB83
:103DC800020203F01133A2EB030303EB2313114A9E
:103DD80003F00F3382FB03121A444FEAE212C2EBDC
:103DE800022248BF0134A3EB020248BFE4B2012A11
:103DF80005DD022A0AD105F08105812D06D1601E54
:103E080002288CBF0020012030BC70470020FBE74F
:103E1800EC1100208180808030B41C7874B11E20A1
:103E2800084D10FB02122A44C91AC8181D28D8BF09
:103E3800147013F8014F0132002CF6D1002030BC69
:103E4800704700BF540C0020014B1888704700BF12
:103E5800D80100200020704700207047002302226C
:103E68000271037043708370C3707047024B1A88E5
:103E78009B780280837070476C8A00083A4B1A78E6
:103E88004AB19A7E19691861012A08D002D3042A16
:103E980000D8704700225A609A60DA60704770B4A0
:103EA80093F82B20B3F9424093ED1A6AD3ED167AB2
:103EB800D3ED1B6A93ED153AB3F94050D3ED125A7E
:103EC80093ED197ADFED293A93ED184AD3ED174AA5
:103ED80003EB420240F6E446128F92B205EE102A36
:103EE80006FB02F2B8EE455A401AC4EB12324FF400
:103EF8007A7101FB02F292FBF5F202FB00F0A5EEEB
:103F0800036A83B01A65E5EE276A9A6007EE900A9D
:103F1800F8EEE77A27EE467AE7EEA35AFCEEC67A81
:103F2800E6EE446ACDED017AF0EE477ABDF804205A
:103F3800C3ED1A6AE5EE247A06FB02F2C4EB1232EC
:103F4800BDEEE57A01FB02F2C3ED1B7A92FBF5F2B6
:103F5800C3ED125ADA645A6083ED117A83ED037A5D
:103F680003B070BC704700BFCC1500202FE33E3172
:103F780070B4344B5A7E012A83B013D00022A3F8C0
:103F88007820A3F87A2093F87E20022A07D1B3F884
:103F98007A10B3F87820A3F88010A3F8822003B031
:103FA80070BC704793F82620D3ED286A93ED234A16
:103FB800D3ED244A93ED297AD3ED277A93ED265A47
:103FC800D3ED255A93F8B01093F8B10093F8B25096
:103FD80003EB420201EB4114128F92B206EE102A53
:103FE800B8EE466A44F6FB76E6EE046AC0EB0030AB
:103FF80004FB0262A6EE247AB2FBF0F2B2FBF5F201
:1040080067EEE67AFCEEE64AA6EEC57A92B2A3F827
:104018008A20CDED014AE6EE257ABDF80410A3F812
:104028007A2004FB0161B1FBF0F1B1FBF5F189B233
:1040380083ED287AC3ED297AA3F88810A3F87810BD
:10404800A1E700BFCC1500200A4BD3F8B41081B10A
:1040580010B4D3F8BC406422002002FB04F25DF8DF
:10406800044BB2FBF1F2C3F8B400C3F8BC00A3F8E8
:10407800B8207047CC1500200B4A136803605368BA
:10408800436030B59368094C83601421002301FB19
:1040980003429579AD0602D51379C37230BD013359
:1040A8000C2BF4D130BD00BF6F8A0008508900087E
:1040B800014B024ADA60FEE700ED00E00400FA0571
:1040C8002DE9F04FDFF8508298F800308FB01BB917
:1040D800884D95F8C0401CB100200FB0BDE8F08FA6
:1040E8000123D5F8C40088F80030FEF799FF802036
:1040F80002F064FC204602F061FC7F4C7F4E0746CC
:10410800D5F8C400FEF792FF23783268BB4240D04E
:1041180001F00CFE7A4AB5F8D630B2F80090DFF814
:10412800FCC1002214464FF0050B4FF0060AEE18AA
:104138001CF8030096F8D810814203F1010704F136
:10414800050115D005EB010E291986F8D80081F86C
:10415800BB321E0A4FF0070381F8B8B281F8BAA241
:1041680081F8BC3281F8B962013206348EF8B8029F
:10417800BBB24B4502F1010232D2632AD7DDA5F862
:10418800D6308CBB0023002088F800300FB0BDE883
:10419800F08F95F8C870002FBCD1D5F8CC30D31A61
:1041A800B3F57A7FB6D9D5F8C4000192FEF738FF87
:1041B800A02002F003FC384602F000FC0746D5F8C0
:1041C800C400FEF733FF95F87E30019A182B7AD099
:1041D800780757D50023C5F8D030C5F8CC2099E723
:1041E8000023A5F8D630CCE7464FA4B23B7803F0BD
:1041F800FF06002BFAD1DFF828A1DFF828915046F6
:10420800FDF724F84846FDF721F803A8FCF7F0FF6E
:104218003D4A3E4BADF8184003A948460392049323
:1042280009960A9607960B960C9605960896FCF73B
:10423800EDFFD9F80030364C43F00103C9F80030DF
:104248001022802303A95046059208930494FCF792
:10425800DDFFDAF80030D5F8C40043F00103CAF8EE
:104268000030D9F8003043F00203C9F80030FEF7F7
:10427800D7FE0123274A3B7093889BB243F0030380
:1042880093807FE707F00507012F2CD0002FA4D1DA
:1042980023785B06A1D5D5F8D010336839B35B1AFB
:1042A800642B9AD9019201F041FD95F87E30019A6C
:1042B800182B92D1B5F8D43001339BB2A5F8D4307D
:1042C800A5F8843089E7237803F04003002B0CBF5E
:1042D8000D211021A5F8803007F00703A5F88610F6
:1042E800A5F8823074E723785906D4D575E7C5F860
:1042F800D03072E7CC15002000000020401C0020C0
:10430800D8010020530C00200C380040DC010020AC
:104318008418002000380040600E0020540C002053
:10432800580002404400024070B5154D154CAB785A
:104338000BBB94F8103503F0F703D4F8C40084F8E5
:104348001035FEF76DFE94F81065042002F036FB78
:10435800304602F033FBD4F8C400FEF767FE297933
:10436800E87801F0C7FC4FF4F0722021064804F009
:10437800DAF9002070BD94F8103543F00803DCE743
:10438800640E0020CC150020540C0020F0B400234B
:104398000C4A0361142702260125522464218360F4
:1043A800836187704360C360436186740580847647
:1043B80083720183C0F80320C0F80B20C0F81320D3
:1043C800F0BC704705040500F8B5264C94F8113583
:1043D800002B46D094F81235002B42D094F81335B0
:1043E80003F0FF07002B3CD1D4F81435C31A002B77
:1043F80037DB1D4B1D491B780625013B05FB0312C6
:104408000A26928AB2FBF6F2D4F8186506F1010E74
:104418000E4405FB031196F822604B8AC4F818E590
:10442800724318441044BEF10E0F88BFC4F81875C3
:10443800C4F81405FDF720FD012384F813350C4B4F
:10444800D4F81C251B8AD4F82015536000234B622E
:104458000B889BB243F001030B80136843F0010300
:104468001360F8BDCC150020001200206C8A0008EB
:104478000C1200202DE9F04F7A4D81B0FDF744FF72
:10448800D5F828450022C5F82425002C00F0AA807C
:10449800237D052B074617D9216A23690B44C31AC4
:1044A8009342B8BF05F5A5610ADBD8E0137D052B5B
:1044B8000AD9136A12691344FB1A002B80F2CF80C1
:1044C80051F8042F002AF1D14FF0010B00231E46AA
:1044D800C5F8243598469A4625E0636A2169227D05
:1044E800FB1AB3FBF1F301331FFA83F912FB09F24C
:1044F8000132013692B2B6B2A4F81890E282904521
:1045080007D2BBF1000F02D1B9F1010F64D990466F
:10451800A246D5F82435013305EB8302C5F82435C6
:10452800D2F828456CB3A268CAB1B4F81690B9F1AC
:10453800000FD2D1216A3846791A9047E8B195F828
:104548005C35002B58D1227D6762013601324FF06D
:104558000103B6B22383E2824FF00109CFE7236A51
:104568002269FB1AB3FBF2F31FFA83F9A4F8189037
:10457800B9F1000F27D1E28AC1E7A4F81890E28ABE
:10458800BDE7D5F8B420D5F8BC30C5F86CA5013224
:104598001E44C5F8B420C5F8BC60BAF1000F28D095
:1045A800DAF8203095F85C25AAF81640FB1ACAF804
:1045B8001C30CAF820709ABBDAF80C30384601B0C3
:1045C800BDE8F04F1847227D12FB09F2013201368F
:1045D80092B2B6B2E28292E7237D062B04BF9046E0
:1045E800A24696E7D5F8B430C5F86C450133C5F84E
:1045F800B43001B0BDE8F08FFDF786FE05F5AC617B
:104608000EC9C01BA1EB511183420144024438BFBB
:104618000346C5F86015C5F86425C5F8683592E7FE
:10462800FDF772FEDAF80C3004469847FDF76CFE89
:10463800DAF82C20DAF82830DAF83010001B90422B
:10464800A3EB53130344014438BF1046CAF828307B
:10465800CAF83010CAF82C0001B0BDE8F08F4FF04E
:10466800000B33E7CC1500202DE9F0413B4ED6F87E
:1046780070550B2D55DC002D6EDDD6F82835984287
:104688004FD0012D39D0D6F82C35984249D0022D7B
:1046980033D0D6F83035984243D0032D2DD0D6F8F4
:1046A800343598423DD0042D27D0D6F83835984275
:1046B80037D0052D21D0D6F83C35984231D0062D7B
:1046C8001BD0D6F8403598422BD0072D15D0D6F8F8
:1046D8004435984225D0082D0FD0D6F84835984251
:1046E8001FD0092D09D0D6F84C35984219D00B2D7A
:1046F80003D1D6F85035984213D0D6F828454CB394
:10470800237D017D8B420FD3154F00243A4605E0E7
:1047180052F8043F53B11B7D8B4207D30134A542A5
:10472800F6DA0020BDE8F0810D4F0024631C9B00E1
:10473800191F2A1B06EB840480463944F818920096
:10474800013503F0D6FFC4F82885C6F87055012056
:10475800BDE8F081024FE9E7CFD0E2E7CC150020B1
:10476800F41A00200D2838B55DD00B285AD8434BD1
:10477800342202FB003021B1C36813B1BDE83840D0
:1047880072E73F4DD5F87045002C4BDDD5F828353C
:1047980098425AD0012C45D0D5F82C35984256D09D
:1047A800022C3FD0D5F83035984252D0032C39D05E
:1047B800D5F8343598424ED0042C33D0D5F8383556
:1047C80098424AD0052C2DD0D5F83C35984246D091
:1047D800062C27D0D5F84035984242D0072C21D056
:1047E800D5F8443598423ED0082C1BD0D5F848352A
:1047F80098423AD0092C15D0D5F84C35984236D085
:104808000A2C0FD0D5F85035984232D00B2C09D04D
:10481800D5F8543598422ED00C2C03D0D5F85835FD
:10482800984204D038BD164BD3F86C05A3E70C2288
:1048380093001448A21A191D014492001844013C1F
:1048480003F057FFC5F8704538BD0022F0E7012294
:10485800EEE70222ECE70322EAE70422E8E7052272
:10486800E6E70622E4E70722E2E70822E0E7092272
:10487800DEE70A22DCE70B22DAE700BFE0010020CE
:10488800CC150020F41A00202DE9F04F83B0484CD5
:10489800484F0190019803685B699847002840F0E9
:1048A8008380DFF818914448D9F80430DFF810E124
:1048B800C3F308034FF00A0A4FF0100C4FF47A754F
:1048C800002B3BD1EFF31183002B37D10168A2688D
:1048D80000BF03689942F9D1DEF8006005FB06F3D2
:1048E8009B1AB3FBF6F305FB013101260091D9F8B9
:1048F8000430C3F30803002B3BD1EFF31183002BE3
:1049080037D10368A16800BF02689342F9D1DEF885
:1049180000B005FB0BF2521AB2FBFBF205FB0323B6
:10492800009A9B1AB3F57A7FE1D3BAF1010AB1D0A4
:10493800D9F80430C3F30803002BC3D0EFF3118276
:104948008CF31288A6682368D90302D501233B603B
:10495800A66803683968D2B282F31188DEF80020AD
:10496800194405FB02F39B1BB3FBF2F305FB013172
:10497800BBE7EFF311888CF31288A1682368DB0387
:1049880044BF3E60A16803683A685FFA88F888F314
:104998001188DEF800801A4405FB08F35B1AB3FBA4
:1049A800F8F305FB0233BBE703B0BDE8F08F00BFA7
:1049B80010E000E03C1C0020401C002000ED00E05E
:1049C800441C0020704700BF704700BF704700BFFD
:1049D800FEE700BFFEE700BFFEE700BF704700BF6D
:1049E800202938B503D80D4621BB284638BD2025D7
:1049F80029461023114A30F8024B22F8044C013B97
:104A080002F10402F7D10120FCF736FB0C490D4AEC
:104A18000B682B440B60136823F4E04323F0400336
:104A28009BB283F0300343F4004343F080031360E8
:104A3800284638BD4B1C5B1089B2DBE78461004017
:104A4800341C0020045C0040B2B170B4541EE4B2BF
:104A58000134002364001E46020F092A02F13005C2
:104A680086BF3732CA54CD54CA1802339C424FEA23
:104A780000105670F0D170BC704700BF30B5144BB1
:104A8800144ADA6083B0142202230024012501A805
:104A98008DF804208DF805308DF806408DF8075004
:104AA80001F0B6FF9DF807308DF805502A228DF8E1
:104AB80006408DF8042033B9074B4FF48062C3F8E1
:104AC800842003B030BD01A801F0A2FF03B030BDBF
:104AD80000ED00E00005FA0500E100E0064B9B7AD6
:104AE80023B9064B01221A6001F0F4BA034B0522E0
:104AF8001A6001F0EFBA00BF7C150020301C0020BE
:104B0800A1490B682DE9F043A04CA14D9BB223802D
:104B180022882B881A40970583B006D54FF6FF5296
:104B28000A60A2780132D2B2A27022881A40160412
:104B380027D4228802F48062134219D1228802F411
:104B48008052134202D103B0BDE8F0838E4A00239D
:104B58004EF6FF7111602373237B052B00F27781DA
:104B6800DFE813F0F600E600E100D600CB00B7005E
:104B7800854A884B4FF6FF315B68116098472B8850
:104B8800DCE70023DFF80082834E844FADF8023063
:104B9800D8F8002090B213044BF6BF7E48F280018B
:104BA800208040F1DC80238803F00F039A0002F193
:104BB800804202F5B842E370002B63D13B689BB298
:104BC800A380A38803F03003E380A38803F4405351
:104BD800A3803B6803EA0E0383F4005383F02003A9
:104BE8000B433B602388D80640F1BB803B689BB2EF
:104BF800ADF80230BDF802301A0500F1D580BDF8D5
:104C080002301904C4D53B68654E40F68F721340D4
:104C1800D6F800803B6098F80830022B0AD0042BA5
:104C280008D0032B00F0F281052B00F0EF81072B51
:104C380000F06382082388F80830FCF72FFA574BF6
:104C48001B68A2884BF6BF71D204A28803EA01034D
:104C580048BF83F480539704E28848BF83F4005325
:104C6800D606E28848BF83F01003900648BF83F059
:104C7800200343F4004343F08003484A9BB2136087
:104C88002B8856E7116889B2ADF80210BDF80210FA
:104C9800090414D4BDF802301A067FF579AFE2781A
:104CA800930003F1804303F5B84306EB82021968C9
:104CB800906948F60F720A401A60804768E71168E1
:104CC80040F68F70013B014056F823301160984739
:104CD800E0E7637B013BDBB26373637B03F0FF02B6
:104CE800002B7FF430AF2F4908684FF6EF7303406D
:104CF80006200B602073226125E72A4A13689BB2BD
:104D080043F0100305200A211360207361731AE72A
:104D1800637B013BDBB26373637B002B7FF413AFD0
:104D2800042323730FE702220323627323730AE722
:104D38001C4D2A684FF6FB7313402B60FFF7CEFE1D
:104D48004FF4164104220123296022732361FAE6F5
:104D58002369002B00F0828005232373F3E62B8858
:104D6800E7E63A680E4E48F60F731A4033683A6021
:104D78001A7A022A00F08080042A7DD0062A00F0E0
:104D8800BD8008221A7258E7445C0040581B002076
:104D9800381C002084010020A08A0008005C004024
:104DA80078150020405C00403B689049904E914A3D
:104DB80040F68F7003403B600968336889B221F080
:104DC80007010A44197A52000929126842D092B29E
:104DD800520002F1804202F5C0421178197092F82F
:104DE800018083F801809088C1B2090241EA10214C
:104DF80059801089C1B2090241EA1021998092892B
:104E0800DA8001211972002A3CD0B8F1060F00F0AF
:104E1800D680B8F1000F7DD1598831B95A6822F48B
:104E28007F42B2F5003F00F02282734F3B68404654
:104E38001B699847032833687ED01A8A4FF6FF719A
:104E48008A4279D002284CD108221A72F5E6062344
:104E5800237378E6DA8893F80180D2E7674D2A68E9
:104E68004FF6FB7313402B60FFF738FE4FF41642E2
:104E780006232A60237366E6FCF732F933681A7A48
:104E88001A72DAE61A7812F07F0258D1B8F1090FCF
:104E980000F01382B8F1050F00F0A581B8F1030FF7
:104EA80000F0B381B8F1010F00F0CE81524F3B689A
:104EB80040465B699847032800F018823368002849
:104EC8007FF45FAF49494E4A096889B221F007016A
:104ED8000A4452000020106030210622E1801A7234
:104EE800ABE6002AB0D093F900100029C0F248813F
:104EF80003214FF440521972A2809EE65A78052A7F
:104F080000F003813C4B1B689B6898473368082274
:104F18001A7292E6B8F1080F40F0CA801A78500663
:104F280083D1384A9A6100205882904733681A8A98
:104F38004FF6FF718A42D4D109221A727DE6012AFE
:104F480000F02D81022AB1D1B8F1010F00F088815B
:104F5800B8F1030FAAD1587947B220F08000820037
:104F680002F1804101F5B841002F0968B4BF01F092
:104F7800300101F44051032898D85888002895D169
:104F8800002993D09B7A002B90D002F1804202F541
:104F9800B842002F1368C0F2E08123F4804323F065
:104FA80070039BB283F4805343F4004343F08003BF
:104FB8001360154B1B689B699847336882E71A781A
:104FC80057067FF432AF9A780B4F012A00F0888198
:104FD800022A00F08881032A7FF428AF3A68526ACF
:104FE800002A9FD14FF0060820E700BF505C004020
:104FF800781500200430002098150020405C0040FF
:1050080002300020390F00089C150020D8F818300D
:10501800B8F810709BB3002F00F09580B8F81420F2
:10502800974228BF17461FFA87F948469847B14A5A
:10503800B14B1268B8F810E0B8F8121092B222F02A
:10504800070213445B00AEEB090E1A6892B27B1C90
:1050580002F1005202F540521FFA8EF789445B10A4
:105068004FEA4202A8F81070A8F8129007D052F838
:10507800041B20F8021B013BF9D1B8F81070002F6F
:1050880068D000214FF440530846A380FBF7F4FF93
:10509800B8F81030B8F81420D6F8008030219A42B9
:1050A800E18053D9002B5BD0052388F80830C2E58E
:1050B800B8F10A0F7FF4B9AE1A7802F07F02012A1C
:1050C8007FF4B3AE9A7A002A3FF4AFAE598800292C
:1050D8007FF4ABAE5A68894F22F47F42B2F5803F25
:1050E8007FF4A4AE58793B689B69984733680028D9
:1050F80000F0408193F8018098E6804B1B68DB68DC
:105108009847D6F80080082395E51A7812F07F02B0
:105118007FF4F8AE93F803C0794840F60F7E036831
:1051280042EA010703EA0E0301323B43042A40F82E
:10513800043BF4D17349744A4CF080030B60136844
:105148001B6A9847DEE6B8F814304BB9032388F891
:10515800083070E5B8F81430D6F80080002BF5D088
:10516800644A062388F808301168684A89B221F031
:1051780007010A445200002030211060E1805AE5FE
:10518800D98801910198824251D95C4A01991268E3
:10519800198292F82C109982FBF7A2FF4DE5B8F11D
:1051A8000B0F7FF483AE554FD9783A6858799369D5
:1051B800984733689A7A002A3FF479AE00287FF43A
:1051C80076AE1A79002A7FF472AE9B78002B7FF4B2
:1051D8006EAE4D4B1B68DB68984733685979DA78AF
:1051E800D9721A736EE693F90320002AFFF6C9AD47
:1051F8009A78002A7FF4C5AD9A88002A7FF4C1AD59
:105208009A7A002A3FF45EAEBBE5DA78012A7FF489
:105218004DAE9A88002A7FF449AE5A7A3A4942F04C
:10522800200209685A72CB69984733684AE6914266
:1052380040F281803149096891F82C60B1B29142FD
:105248006FD900222272A6E7DA78012A7FF42EAEFF
:105258009A88002A7FF42AAE5B7A9B067FF526AEF1
:1052680003F0ACF900287FF421AE33682AE693F8FE
:10527800008018F07F084DD0B8F1010F60D0B8F168
:10528800020F4BD193F8058008F00F018A0002F154
:10529800804202F5B84218F0800F126814BF02F07D
:1052A800300202F44052032938D818F0700835D17A
:1052B800002A3FF4BAAD164A34E6DA788A423FF655
:1052C800F5AD997800297FF4F1AD998800297FF42C
:1052D800EDAD0D499A720B685B6898473368F1E544
:1052E8003A68D2697CE63A68126A79E63368092234
:1052F8001A72A2E4505C0040043000209815002087
:10530800005C00404C5C00409C15002002300020EE
:10531800850E00089A88002ACDD086E54FF000084F
:1053280083E592FBF6F006FB1022002A7FF433AFE8
:10533800012222722FE7104A126892F82C102AE7ED
:105348000D4F58793B689B699847336800287FF46C
:10535800D1AE9A7A002AAED1CCE623F4E04323F00A
:1053680040039BB283F0100343F4004343F08003EF
:1053780013601EE6014AD5E598150020110F0008B4
:10538800FF207047012380F849307047002280F8D9
:10539800492001F023B990F84820531C0244DBB29D
:1053A80080F8483082F8341090F849200AB1132B5D
:1053B80001D901F013B970472DE9F04F87B00A23DE
:1053C800BD4DBE4FBE4CBF4E04900393BE4B1978E3
:1053D8009868C1F34001FDF72FFEBB4B1978586858
:1053E800C94301F00101FDF727FE05230293B64BDF
:1053F800DFF8D8929868FDF709FEB34B5868FDF7B7
:1054080005FE4FF0320A4FF0100C4FF47A70D9F8BD
:105418000430C3F30803002B40F0CB81EFF3118372
:10542800002B40F0C6812968A26800BF2B6899420A
:10543800F9D1D7F800E000FB0EF39B1AB3FBFEF39B
:1054480000FB01314FF0010E0191D9F80430C3F38C
:105458000803002B40F03C81EFF31183002B40F050
:1054680037812B68A16800BF2A689342F9D1D7F821
:1054780000B000FB0BF2521AB2FBFBF200FB032355
:10548800019A9B1AB3F57A7FDFD3BAF1010ABED12C
:105498008D4BDFF838929868FDF7B8FD8A4B58684D
:1054A800FDF7B4FD4FF0320A4FF0100C4FF47A704C
:1054B800D9F80430C3F30803002B40F05D81EFF303
:1054C8001183002B40F058812A68A16800BF2B681F
:1054D8009A42F9D1D7F800E000FB0EF35B1AB3FB50
:1054E800FEF300FB02324FF0010E0192D9F80430AE
:1054F800C3F30803002B40F0C380EFF31183002BA4
:1055080040F0BE802B68A16800BF2A689342F9D199
:105518008846396800FB01FBABEB0808B8FBF1F8DB
:1055280000FB0383019A9B1AB3F57A7FDED3BAF1A5
:10553800010ABDD1029B013B13F0FF0302937FF4E4
:1055480056AFDFF888A14FF4FA784FF0100C4FF4FB
:105558007A70DAF80430C3F30803002B40F0468170
:10556800EFF31183002B40F041818E462A68A16831
:1055780000BF2B689A42F9D10B4671469E4600FB44
:1055880001F3A3EB0E0EBEFBF1F100FB02124FF08C
:10559800010E0192DAF80430C3F30803002B40F03F
:1055A800CF80EFF31183002B40F0CA802B68A168ED
:1055B80000BF2A689342F9D18946396800FB01FB8C
:1055C800ABEB0909B9FBF1F900FB0393019A9B1AAC
:1055D800B3F57A7FDED3B8F10108BAD1049BFF2B6B
:1055E80040F03E814FF47A7ADFF8E09050464FF071
:1055F800100CD9F80430C3F30803002B40F01381D2
:10560800EFF31183002B40F00E812968A26800BFD8
:105618002B689942F9D1D7F800E000FB0EF39B1AEA
:10562800B3FBFEF300FB01314FF0010E0191D9F8F5
:105638000430C3F30803002B66D1EFF31183002B6A
:1056480062D12B68A16800BF2A689342F9D1D7F8C4
:1056580000B000FB0BF2521AB2FBFBF200FB032373
:10566800019A9B1AB3F57A7FE1D3BAF1010AC0D146
:10567800039B013B03937FF4A9AE07B0BDE8F08F0D
:10568800EFF311818CF31288A2682368DB0344BF0F
:10569800C6F800E0A2682B68D6F80080C9B281F38A
:1056A80011883968434400FB01F8A8EB0208B8FBED
:1056B800F1F800FB038335E7401C0020441C002060
:1056C80010E000E03C1C00206C1B002000ED00E016
:1056D800EFF311888CF31288A1682368DB0344BFB9
:1056E800C6F800E0A1682B6832685FFA88F888F38A
:1056F8001188D7F800801A4400FB08F35B1AB3FB43
:10570800F8F300FB0233BBE6EFF311888CF3128841
:10571800A1682368DB0344BFC6F800E0A1682B68D2
:1057280032685FFA88F888F31188D7F800801A443D
:1057380000FB08F35B1AB3FBF8F300FB02338FE7B7
:10574800EFF311818CF31288A2682368DB0344BF4E
:10575800C6F800E0A2682B68D6F80090C9B281F3B9
:10576800118839684B4400FB01F9A9EB0209B9FB20
:10577800F1F900FB039329E7EFF311818CF3128809
:10578800D4F808E02368DA0303D501233360D4F89A
:1057980008E02B683268C9B281F3118839681A4465
:1057A80000FB01F3A3EB0E03B3FBF1F300FB0232A2
:1057B80099E6EFF311828CF31288D4F808E0236895
:1057C800D90303D501233360D4F808E02B68316886
:1057D800D2B282F311883A68194400FB02F3A3EBB2
:1057E8000E03B3FBF2F300FB01312BE6EFF311815B
:1057F8008CF31288D4F808E02368DA0303D5012370
:105808003360D4F808E02B683268C9B281F3118894
:1058180039681A4400FB01F3A3EB0E03B3FBF1F361
:1058280000FB0232B3E6EFF311828CF31288D4F84E
:1058380008E02368D90303D501233360D4F808E0CE
:105848002B683168D2B282F311883A68194400FB98
:1058580002F3A3EB0E03B3FBF2F300FB0131E3E623
:10586800944B19789868C1F34001FDF7E5FB914B1B
:1058780019785868C94301F00101FDF7DDFB049B65
:10588800CDF80880013305938A4BDFF82C9298688D
:10589800FDF7BCFB874B5868FDF7B8FB4FF0FA0AD9
:1058A8004FF0100C4FF47A70D9F80430C3F30803A2
:1058B800002B40F0E280EFF31183002B40F0DD80F5
:1058C8002968A26800BF2B689942F9D1D7F800E08F
:1058D80000FB0EF39B1AB3FBFEF300FB01314FF004
:1058E800010E0191D9F80430C3F30803002B40F0EE
:1058F8008B80EFF31183002B40F086802B68A16822
:1059080000BF2A689342F9D1D7F800B000FB0BF228
:10591800521AB2FBFBF200FB0323019A9B1AB3F560
:105928007A7FDFD3BAF1010ABED1624BDFF88891E2
:105938009868FDF76BFB5F4B5868FDF767FB4FF006
:10594800FA0A4FF0100C4FF47A70D9F80430C3F308
:105958000803002B74D1EFF31183002B70D1296851
:10596800A26800BF2B689942F9D1D7F800E000FB84
:105978000EF39B1AB3FBFEF300FB01314FF0010E4F
:105988000191D9F80430C3F308030BBBEFF311837B
:10599800F3B92B68A16800BF2A689342F9D1D7F8F8
:1059A80000B000FB0BF2521AB2FBFBF200FB032320
:1059B800019A9B1AB3F57A7FE3D3BAF1010AC4D1ED
:1059C800029B059A01339A4202937FF45DAF09E680
:1059D800EFF311888CF31288A1682368DB0344BFB6
:1059E800C6F800E0A1682B6832685FFA88F888F387
:1059F8001188D7F800801A4400FB08F35B1AB3FB40
:105A0800F8F300FB0233D3E7EFF311888CF3128825
:105A1800A1682368DB0344BFC6F800E0A1682B68CF
:105A280032685FFA88F888F31188D7F800801A443A
:105A380000FB08F35B1AB3FBF8F300FB02336CE7D7
:105A4800EFF311828CF31288D4F808E02368D903A5
:105A580003D501233360D4F808E02B683168D2B24B
:105A680082F311883A68194400FB02F3A3EB0E0392
:105A7800B3FBF2F300FB013180E7EFF311828CF303
:105A88001288D4F808E02368D90303D501233360CA
:105A9800D4F808E02B683168D2B282F311883A68EA
:105AA800194400FB02F3A3EB0E03B3FBF2F300FB74
:105AB800013114E76C1B002000ED00E010B5FBF786
:105AC80083FB01280CD14FF4302400E04CB1FBF7E4
:105AD8007BFB012804F1FF34F8D0002C08BF052017
:105AE80010BD052010BD2DE9F0411C4C23691BB9E0
:105AF800256985B3EFB201E001273D460023267DE5
:105B08001946E21832440133DBB2127E4254AB42EA
:105B18001946F6D323695B1B2361D4F810803E44F1
:105B28002675B8F1000F13D140210320FBF780FA46
:105B38000B4A84F81480136823F4804323F070031D
:105B48009BB283F4405343F4004343F08003136053
:105B58002846BDE8F081267D2F46DBE76C1B002038
:105B68000C5C0040F8B50568037B2A6802269E4055
:105B780032420DD1296804229A40114218BF6A6046
:105B88002968082202FA03F3194218BF6B60F8BDAE
:105B98001749184A0B684FF6FE7423400B601389A7
:105BA8009F07FCD5134B1A891406FCD41B89D90707
:105BB80018D411490F4A0B684FF6FE773B400B602B
:105BC8006E60938823F0030304461B040B481B0CE8
:105BD80093800068FDF72AFA094A2568237B00218B
:105BE8001170C7E7034B9A891A89D207E1D5FAE7FA
:105BF800440002400038004058000240901600203F
:105C0800530C002010B490E80600047B406902237E
:105C1800A3404B6013685DF8044B4FF6FE710B40D0
:105C28001360FCF751BD00BF2DE9F84F2A4A1378DD
:105C380003F0FF04002BFAD1DFF8ACA0DFF8AC804A
:105C4800DAF80000DFF8A890244F012388F8003024
:105C5800FDF7E6F9052000F0B1FE204600F0AEFEA3
:105C6800062000F0ABFE204600F0A8FE99F8005090
:105C7800042045F0010500F0A1FE284600F09EFE34
:105C88003B888BB1164D174E95F801B0072000F0F0
:105C980095FE584600F092FE3B8815F8012F06F84D
:105CA800012F01349C42EFDB072000F087FEFF2024
:105CB80000F084FE99F80040042000F07FFE2046A2
:105CC80000F07CFEDAF80000FDF7B0F9002388F850
:105CD8000030BDE8F88F00BF530C0020D801002029
:105CE800530C0020A316002090160020600E002000
:105CF800DC1A002070B50C4EC1F1030545EA800599
:105D08003068FDF78DF9EDB21024E0B200F056FED0
:105D18000134284600F052FE202CF6D13068BDE848
:105D28007040FDF783B900BF90160020F8B5394CD4
:105D38002068FDF775F9384B1B78012B5BD048D3E9
:105D4800022B3ED1354D08232B704FF4C373344ECC
:105D5800344F338002210020FFF7CCFF2068FDF785
:105D68005FF92D78002000F029FE284600F026FE75
:105D78002D4B1D78022000F021FE284600F01EFE63
:105D88002A4B1D78032000F019FE284600F016FE65
:105D9800274B1D780420054300F010FE284600F02C
:105DA8000DFE2068FDF742F932882248002102F0F2
:105DB800BAFC3B7863B1204B1B7813B300233B70CC
:105DC800F8BD164D2B785B06BFD54FF4F073BEE7D0
:105DD800F8BDA02000F0F2FD002000F0EFFD00F07B
:105DE8000603022B0D4D03D000F0050001280DD04D
:105DF80008232B70A9E7094D48232B704FF4F07343
:105E0800A5E7FFF711FF00233B70F8BD48232B706F
:105E1800DBE700BF90160020941600200000002049
:105E2800D801002050040020BC090020BD09002032
:105E3800DC1A0020A4160020600E002070B50F4C5C
:105E48000F4DC0EBC00004EB80046869266930433D
:105E5800686182B09209667BA1600025012101A8D2
:105E680063618DF804608DF805208DF806508DF873
:105E7800071000F0CDFD02B070BD00BF3400002057
:105E8800001002400348D0F83C3113B100F59A7075
:105E980018477047340000200348D0F8203113B168
:105EA80000F58C7018477047340000200348D0F87C
:105EB80004310BB1FC301847704700BF3400002094
:105EC8000348D0F8E8300BB1E0301847704700BFFE
:105ED800340000200348D0F8CC300BB1C430184748
:105EE800704700BF340000200348D0F8B0300BB131
:105EF800A8301847704700BF340000200348D0F886
:105F080094300BB18C301847704700BF3400002024
:105F18000248836F0BB17030184770473400002077
:105F28000248C36D0BB15430184770473400002045
:105F38000248036C0BB13830184770473400002012
:105F48000248436A0BB11C301847704734000020E0
:105F58000248836803B11847704700BF3400002027
:105F6800F8B5574C0601A7190546387A00F008FD20
:105F78003B7A03F01F015B090122022B02FA01F2AE
:105F880078D0032B71D0012B67D0A319013518796C
:105F9800FCF7EAFBEDB2074610B11223C571837115
:105FA800A3195879FCF7E0FB10B11323C57183716D
:105FB800A3199879FCF7D8FB10B11423C571837124
:105FC800A5190E21EA793846FCF792FC6879FCF7A6
:105FD800CBFBEA790E21FCF78BFCA879FCF7C4FB14
:105FE800EA790E21FCF784FCA359364A934251D032
:105FF800354A934259D0354A934240D03444227BA3
:10600800002A2FD1012002249A8822F480521204F7
:10601800120C9A80998889B241F4805199801A8823
:1060280002F4415242F44572024322431A809A888C
:1060380022F470621204120C42F4E0629A809A8B85
:1060480022F400621204120C07219A8319821A881A
:1060580092B242F040021A80F8BD1D4B996A0A4379
:106068009A6292E700200446CEE7194B19690A4361
:106078001A618AE7164BD9680A43DA6085E702F5A0
:10608800EA32116941F400411161116921F40041BA
:106098001161B3E702F56042D16841F48051D160E3
:1060A800D16821F48051D160A8E702F5EC3211697A
:1060B80041F480411161116921F4804111619DE72A
:1060C800481C00200030014000380040003C0040DF
:1060D800001002401749184B184A194810B4D1F853
:1060E800884044F47004C1F888401C6844F00104F6
:1060F8001C605C6822405A601A6822F0847222F49C
:1061080080321A601A6822F480221A605A6822F4CF
:10611800FE025A60DA6A22F00F02DA621A6B002471
:1061280010404FF0006218639C608A605DF8044B71
:10613800704700BF00ED00E0001002400CC07FF87F
:10614800CCFC00FF014B1868704700BF7C1B002087
:10615800012070477047704708B103487047034BE8
:106168001B6808221A8270476804002078150020EE
:10617800F2E709B10220704701288CBF02200020F5
:1061880070470C4B1B68DA78042A07D8598A38B14B
:10619800094B03EBC2039868084470470020704716
:1061A80010B4054C04EBC2025DF8044B9289511AF5
:1061B800198270477815002068040020064B1B6878
:1061C8005A8A18B1054B986A104470470349898D5B
:1061D8008A1A1A82704700BF7815002068040020C8
:1061E800064B1B685A8A18B1054B186B1044704748
:1061F8000349898E8A1A1A82704700BF78150020D1
:1062080068040020074B1B681B7803F07F03212BD1
:1062180001D00220704700F0DF00022814BF0220DE
:106228000020704778150020212804D02028034634
:1062380011D0022070470F4B1A68137803F07F03C0
:10624800212BF6D10C4910B50024916154822046C7
:106258008847204610BD074A1268117801F07F016F
:10626800212903D0054A02201370704703480449C6
:106278000370E8E778150020796100082C1C0020DD
:10628800616100087047034B1A78202A04BF002276
:106298001A7070472C1C0020014B04225A6070476A
:1062A8002C1C0020034B9B7A13B1034B05225A6028
:1062B800704700BF7C1500202C1C00200D4A0E4B97
:1062C80012680E4992B222F0070213445B001B6861
:1062D800C3F309030B600B689BB201335B1007D053
:1062E8000749084A52F8040B21F8020B013BF9D17F
:1062F800704700BF505C00401E3000207C1B00200F
:10630800841B002020620040014B00229A607047E5
:106318002C1C00202DE9F0410F4D6B681746B3B1D6
:106328006B68052B13D10D4ED6F800800C46002F54
:106338000DDDAB686BB939462046FEF751FB336873
:10634800A3EB0803322BA7EB00070444EFD9BDE801
:10635800F0810020F3E700BF2C1C0020401C002027
:1063680007B501A8FFF7BFFB0028FAD09DF8040085
:1063780003B05DF804FB2DE9F04F6B4BDFF8D081DB
:106388001A686A4DDFF8CCB1DFF8CC9168496948E2
:10639800DFF8C8A1684F83B00024C02353729472F9
:1063A800D4720193C8F800402A6802EA0B0242F44A
:1063B800007292B22A602A6802EA090292B248F28E
:1063C800800682F0100232432A60D8F8002092B288
:1063D80022F007021144490040220A60D8F8001050
:1063E800009289B221F0070101F1005101F54051F5
:1063F80049004FF0800EC1F800E0D5F800E090F8B1
:106408002C1040F60F6000EA0E003043286020464A
:10641800FAF70EFE29684948DFF844E1019B009A23
:1064280001EA0A0189B281F44051314329600168C7
:1064380001EA0B0189B20160D8F8001089B221F095
:1064480007018E444FEA4E0E1146CEF8003003681D
:106458003B4ADFF810E103EA09039BB283F020030B
:1064680033430360036803EA0A0333439BB20360C0
:106478001368344803EA0B0343F4C0639BB2136008
:10648800D8F800309BB223F007039E444FEA4E0E23
:106498004FF48073CEF80030136803EA0A033343DD
:1064A8009BB21360136803EA09039BB283F02003CD
:1064B800334313603B6803EA0B0B1FFA8BF33B6013
:1064C800D8F800309BB223F00703184440004FF47B
:1064D800887303600320FAF7ABFD3B6803EA0A03FD
:1064E8009BB283F4405333433B603B6803EA0903A0
:1064F80033439BB22A4620463B60314640F60F752F
:10650800136840EA01042B4001302343042842F871
:10651800043BF5D10C490D4B8020012208605A60DC
:1065280003B0BDE8F08F00BF78150020005C004084
:1065380004300020840100200C5C0040045C004012
:10654800085C00401C3000204C5C00402C1C0020E3
:10655800505C00408F89FFFFBF8FFFFF8FBFFFFF99
:106568000830002010300020F8B5134A134B10688B
:106578001B68C0180AD0124B12491C680822FEF783
:1065880063FA204604221049FEF75EFA0F4B104AC0
:106598001F68104C10490023BB724FF416400126A7
:1065A8004FF4E055888116601360236015602360FE
:1065B80010604B60F8BD00BFACF7FF1FB4F7FF1FBA
:1065C800B0F7FF1FA2040020B204002078150020B5
:1065D800405C0040445C00402C1C00202DE9F04148
:1065E80090F84850002380F848300DB3154E726873
:1065F8000AB37268052A21D1134FD7F8008000F139
:106608003404B36893B929462046FEF7E9F93B6894
:10661800A3EB0803322BA5EB0005044401D8002D99
:10662800EFD1B5FA85F04009BDE8F0810020EEE72A
:106638000120BDE8F0811046BDE8F0811846BDE8AC
:10664800F08100BF2C1C0020401C0020024B4FF49E
:1066580080221A60704700BF140401402DE9F047FA
:106668003E4ADFF800E13E484FF00A0C10254FF48F
:106678007A740127DEF80430C3F30803002B50D1E5
:10668800EFF31183002B4CD15668816800BF536823
:106698009E42F9D1D2F8088004FB08F35B1AB3FBD9
:1066A800F8F304FB063ADEF80430C3F30803EBB949
:1066B800EFF31183D3B95368D0F8088000BF51684D
:1066C8008B42F8D1D2F8089004FB09F1A1EB080835
:1066D800B8FBF9F804FB0383A3EB0A03B3F57A7F4D
:1066E800E1D3BCF1010CC5D1BDE8F087EFF3118807
:1066F80085F3128886680368DB0344BF17608668E1
:10670800516813685FFA88F888F31188D2F808800E
:106718000B4404FB08F1891BB1FBF8F104FB0313DC
:10672800DAE7EFF3118185F31288D0F8088003685F
:10673800DE0344BF1760D0F8088053681668C9B2F2
:1067480081F3118891681E4404FB01F3A3EB08034D
:10675800B3FBF1F304FB063AA5E700BF3C1C00209D
:1067680010E000E000ED00E02DE9F0473E4ADFF8D8
:1067780000E13E484FF0190C10254FF47A740127B8
:10678800DEF80430C3F30803002B50D1EFF3118374
:10679800002B4CD15668816800BF53689E42F9D1DE
:1067A800D2F8088004FB08F35B1AB3FBF8F304FB88
:1067B800063ADEF80430C3F30803EBB9EFF31183AC
:1067C800D3B95368D0F8088000BF51688B42F8D11C
:1067D800D2F8089004FB09F1A1EB0808B8FBF9F816
:1067E80004FB0383A3EB0A03B3F57A7FE1D3BCF17F
:1067F800010CC5D1BDE8F087EFF3118885F3128845
:1068080086680368DB0344BF1760866851681368AD
:106818005FFA88F888F31188D2F808800B4404FBE3
:1068280008F1891BB1FBF8F104FB0313DAE7EFF376
:10683800118185F31288D0F808800368DE0344BF0D
:106848001760D0F8088053681668C9B281F31188B8
:1068580091681E4404FB01F3A3EB0803B3FBF1F3B7
:1068680004FB063AA5E700BF3C1C002010E000E04E
:1068780000ED00E02DE9F0473E4ADFF800E13E4830
:106888004FF0C80C10254FF47A740127DEF8043055
:10689800C3F30803002B50D1EFF31183002B4CD125
:1068A8005668816800BF53689E42F9D1D2F80880C3
:1068B80004FB08F35B1AB3FBF8F304FB063ADEF8B3
:1068C8000430C3F30803EBB9EFF31183D3B953686A
:1068D800D0F8088000BF51688B42F8D1D2F80890F0
:1068E80004FB09F1A1EB0808B8FBF9F804FB0383E2
:1068F800A3EB0A03B3F57A7FE1D3BCF1010CC5D150
:10690800BDE8F087EFF3118885F31288866803687D
:10691800DB0344BF17608668516813685FFA88F81C
:1069280088F31188D2F808800B4404FB08F1891B0E
:10693800B1FBF8F104FB0313DAE7EFF3118185F3F8
:106948001288D0F808800368DE0344BF1760D0F8C7
:10695800088053681668C9B281F3118891681E448B
:1069680004FB01F3A3EB0803B3FBF1F304FB063AC2
:10697800A5E700BF3C1C002010E000E000ED00E0AF
:1069880000F01F0240090123022803FA02F30ED087
:10699800032807D0012800D07047074A51690B43E4
:1069A80053617047044AD1690B43D3617047024A67
:1069B80091690B43936170470010024040F2E9333C
:1069C800104900E0B3B10A89013B12F0020F9BB2F3
:1069D800F8D00D4B0B49187040F2E93300E04BB189
:1069E8000A89013B12F0010F9BB2F8D0064B1878C8
:1069F800C0B27047054AD38C01339BB2D384D08C84
:106A0800C0B27047003800400C3800403C1C0020E1
:106A180030B40C4B0178DA6843780B4CD243C2F39C
:106A28000222C2F10402934060181B0101F01F0505
:106A380001224909DBB2AA4080F8003344F821203A
:106A480030BC704700ED00E000E100E000231B6867
:106A5800FFDE00BF03685A1C0260197070472DE9F9
:106A6800F341056906460F467DBBD0F80080C8F3A0
:106A78000A0323B30023D6F800800193FFF71EF81A
:106A8800042819D1214C236943F001032361BBB2C7
:106A9800A8F80030FFF712F804282ED108F10203F5
:106AA8000193019B3F0C1F80FFF708F82369042816
:106AB80023F00103236125D06FF0010505E0FEF7FF
:106AC800FDFF042805D04FF0FF35284602B0BDE889
:106AD800F0810E4C236943F002032361C4F814804B
:106AE800236943F040032361FEF7E8FF2369042884
:106AF80023F002032361BDD0E5E7236923F00103F6
:106B08002361D9E7336804333360DEE700200240AD
:106B180070B5448806460D46C4F30B04224600218E
:106B2800284601F000FE3369094A934209D3094A0D
:106B3800934206D2224628461946BDE8704001F025
:106B4800CDBD23B121462846BDE87040184770BD29
:106B58008C8D0008C68D0008024A136823EA0000DD
:106B6800106070472C0C0020002870B51EDB092827
:106B7800044620DD012303EB83035B00B0FBF3F243
:106B8800092AF8D87BB10E4EB4FBF3F00928CCBF24
:106B980057223022A6FB03E5024403FB1044EB080E
:106BA80001F8012BF0D100230B7070BD2D230B7061
:106BB80040420131DBE7303001F8010BF3E700BF59
:106BC800CDCCCCCC884230B44FF001042ED301FB9D
:106BD80004F4B0FBF4F58D42F9D284B1AAB901E00E
:106BE800B0FBF4F5092DCCBF572230222A4404FB10
:106BF800150003F8012BB4FBF1F4002CF0D10022AE
:106C08001A7030BC7047B0FBF4F5092DCCBF3722A1
:106C180030222A4404FB150003F8012BB4FBF1F4DD
:106C2800002CF0D100221A7030BC70470546002AAB
:106C3800EBD1D7E7FAB170B48E18044603E0101A06
:106C480014D1B14214D014F8012BA2F14103192B2D
:106C580011F8013BA3F1410598BF2032192D03F12A
:106C68002000ECD9D01A01D1002BEAD170BC7047B2
:106C7800002070BC70471046704700BF4FF0FF32CD
:106C8800FFF7D8BFA0F16103192B98BF20387047D0
:106C9800A0F14103192B98BF20307047202805D058
:106CA800093804288CBF0020012070470120704754
:106CB800613819288CBF00200120704741381928F5
:106CC8008CBF002001207047303809288CBF002075
:106CD80001207047A0F13003092B07D920F02000CC
:106CE800413819288CBF00200120704701207047C7
:106CF8000368591C1A46016012F8021B0260587892
:106D080041EA0020704700BF38B5044600681546C0
:106D180001F0E4FC22682A44226038BD03685A1C4A
:106D2800026010B4197003680A0A5C1C04601A70C7
:106D380003680A0C5C1C04601A700368090E5A1C6C
:106D4800026019705DF8044B704700BF03685A1C55
:106D5800026019700368090A5A1C026019707047AA
:106D68000A44914214D030B40139551E41F221022F
:106D780011F8014F082380EA042004044CBF82EA7A
:106D880040004000013B80B2F7D18D42F0D130BCC9
:106D9800704770B5154C2378A52B24D16378BE2B8A
:106DA80021D1214602224FF6FF70FFF7D9FF104E7E
:106DB800023422884AB1A518B54214D2052A12D93C
:106DC8002146FFF7CDFF2C46F3E721460222FFF7C5
:106DD800C7FF0222A118FFF7C3FF41F60F53C31ADA
:106DE8005842584170BD002070BD00BF00F0030834
:106DF800000004082DE9F041804B814C1D885B8818
:106E0800E278EB1A83EAE3719542A1EBE37149D387
:106E18002378AB4246D37B4A1378DE1E012E40F21C
:106E28009D80794E3678022E00F08E80012B6DD031
:106E380077D3022B04D19188A94201D20123137080
:106E4800E17A002948D02189002945D06F4D2D7855
:106E5800002D41D06E4D9FED6F6AD5ED026A07EEA9
:106E6800901AF8EEE66AB8EE677AF8EEE77A77EE07
:106E7800666A66EE866A86EEA77AFDEEC77A17EE30
:106E8800901A0029C0F29380642900F3B480002985
:106E980000F08D80C9B2257B8D422CBF01250025CD
:106EA80055701AE0B5EB420FB5DC564A1378DE1E72
:106EB800012E40F298800229B3DC534BDFF84CE1F5
:106EC8001F7800260323022F8EF8006056809680D4
:106ED80013705370B4D139E055782479632C03D8F2
:106EE800022B117A66D029B9AB4238BF2B461374EE
:106EF800BDE8F081D168401A4749884260DDAB425D
:106F080038BF2B4654721374BDE8F0819188667BB4
:106F1800891B8D420CDD5188A94291D20023137040
:106F28008EE75688637BF61AB54287DD002387E72C
:106F38000223137084E70229BFDD334B1B78022B31
:106F48004FF004037FF47CAF304E3678334F02297C
:106F5800CCBF00210121F980BE8067E702293FF7F5
:106F680060AF267895FBF6F6771C082F274BDFF8DD
:106F780098C0A67894F801E09CF800C0A8BF08273C
:106F88001F70BBB216FB03F61EFB03FEB6B200234E
:106F98004FF06408BCF1020F5680A2F804E01370A9
:106FA8005370D36082F80980BCD13EB2CEE7022587
:106FB800557092E700299DD10126D06016720846C7
:106FC800C4F16404164900FB04F081FB0041C017BA
:106FD800A0EBA150AB4200F1640038BF2B465072C1
:106FE8001374BDE8F081032BA5D1074E3678022E25
:106FF8007FF426AFA8E764214DE700BF44160020C0
:10700800E0150020781C00204A160020CC1500202E
:10701800D01500200000C8427F9698004C1600202A
:107028006BCA5F6B1F4B204870B5342201250021C5
:107038001D7001F078FB1D4A1D491E4C1E48002397
:107048000B601360FDF710FB29460520FDF78AFB4E
:107058006579291C4FF0070018BF0121FDF782FB55
:10706800A679311C4FF0080018BF0121FDF77AFB03
:10707800A37A0BB9E17A19B195B9311C18BF01216E
:107088000920FDF76FFB0D4B59690A20C1F34051E8
:10709800FDF768FB01210B20BDE87040FDF762BBDE
:1070A8000121EDE7281B0020F41A00203C1B0020DA
:1070B800F01A0020E0150020E0010020781C0020D4
:1070C800034613F8012B002AFBD1181A0138704720
:1070D800430803F05533C01A830803F0333300F034
:1070E8003330184400EB101000F00F3000EB002094
:1070F80000EB0040000E704711481249026800601A
:107108008A4218D0002103E00F4B5B5843500431EA
:107118000E480F4B42189A42F6D30E4A02E000235B
:1071280042F8043B0C4B9A42F9D3FEF7D3FF00F028
:1071380019F87047FEE70948D0F800D040680047C2
:10714800FC9F0020EFBEADDEC68D000800000020C9
:10715800BC040020BC040020901D002000D8FF1FA4
:10716800FEE700002DE98048BB4BBC4AA1B0196876
:10717800914200AF00F0EB86B949BA4B00224FF4B8
:107188007000C1F888003A627A621A6842F4803264
:107198001A6003E03A6AB2F5A04F09D01A6802F4FF
:1071A80000327A623A6A01323A627A6A002AF1D087
:1071B800AC4B1B6813F4003318BF01237B627B6A56
:1071C800012B00F09986A64CA64BA74AE2605A6AA2
:1071D8005A6ADFF8E89242F080725A625A6942F4B9
:1071E800FC025A6100250322012307F1300141F610
:1071F800FF764FF090407D633E6387F8342087F830
:107208003630FAF7B7F84FF6FF7307F130019748B1
:107218003B63FAF7AFF807F130019548954EFAF756
:10722800A9F807F130019448FAF7A4F807F13001FA
:107238009248FAF79FF807F130019148FAF79AF85F
:1072480007F13000FAF7A2F93B6B8E498E4A8F4856
:10725800A1FB03139B0C3360F0210723506084F8D3
:10726800231095601360FBF7A5FAFFF792FD884D90
:10727800002800F06E85874CA94523D2DFF83C92A0
:10728800DFF83C82464633889B46F2188BB1A2420F
:107298000FD2052B0DD9B9F800307188C3F30B0351
:1072A800994200F01581164633889B46F218002B48
:1072B800EDD1D9F80410484609F11409FFF728FC64
:1072C800A945DFD3FCF71AFD002800F01B81012037
:1072D800FFF742FC0820FFF73FFC4020FFF73CFC8B
:1072E8008020FFF739FC4FF40070FFF735FC4FF4AE
:1072F8008060FFF731FC4FF40050FFF72DFC4FF48E
:107308008040FFF729FC4FF48030FFF725FC4FF44D
:107318000030FFF721FC4FF48020FFF71DFC5E488A
:107328005E4CDFF8A0A15E4DDFF89C91FFF714FCDE
:107338004FF00070FFF710FC4FF08060FFF70CFC77
:107348004FF00060FFF708FC4FF00050FFF704FC17
:10735800544A554B554910781B78554A087052487D
:107368001268E178CAF8002043F00103037029701D
:107378004FF001080526CB4614F8010B002840F011
:10738800E880CBF800005B4608F101080433B8F147
:10739800040F9B46F0D12978D9F80000454CC94321
:1073A80001F00101FBF748FE2978D9F8040081F0C3
:1073B8000201C1F34001FBF73FFE2978D9F8080024
:1073C80081F00401C1F38001FBF736FE01210220A0
:1073D800FBF73CFEFBF724FF6420FAF7F7FEFAF709
:1073E8005BFD2320FBF7C0F9C4F8C00418B11122D3
:1073F80000238271C3710121FBF74CFCD4F8C0044F
:107408002C4CDFF8C880FBF70BFE2B4B224603F110
:10741800200B19201A21002503F1110C08EB050691
:1074280003F1140EC7F814C03E6131B13E6996F8F5
:107438000AC08C4508BF82F85C1028B118F80510FE
:10744800814208BF82F85D00786986455ED010F8F1
:10745800011B7861C078E8E7FC9F0020EFBEADDE35
:1074680000ED00E0001002400005FA0500040048A5
:1074780000080048441C0020000C00480010004888
:107488000014004883DE1B4310E000E03F190100B0
:107498008C8D00080000040820001000A8110020AE
:1074A8006C1B0020240C0020221000204A1600200B
:1074B8002C0C0020BC04002040870008388C0008F1
:1074C80002F003088C1C0020701B0020CC11002047
:1074D800737999077FF4E7AED9F8041096F804A0F9
:1074E8004846FFF715FBB9F80030BAEB133F20D038
:1074F80009F11409A945FFF4C5AEFCF7FFFB002804
:107508007FF4E5AE5248FCF741FFE0E6B2F85C10C4
:1075180029B15049936541F8252002F518729B4519
:1075280026D093F8205093F8301093F83400203385
:1075380072E7B9F80230D9F80400ABF10602C3F3D8
:107548000B039A4206F10601A8BF1A4601F0C6F8D5
:10755800CEE7FBF709F90121CBF800005FFA88F3C1
:1075680018B18671C371DBF80000FBF793FB0AE7DB
:10757800FCF7A6FB0020FEF7F3FCDFF8E8B0364D79
:10758800DFF8E4800120FEF7EBFC00212246002D05
:1075980043D01BF90B6C314818F806C07A60B30069
:1075A80008EB060403EB060EA478BB604FEA8E03D3
:1075B80018443C61D318294CFB60ABF1030344F831
:1075C8002E107B6141608160C160016164467B6906
:1075D80013F8012B7B61A24230D07B699A783B6912
:1075E8009A4222D07B695B45F1D1BB687A68334403
:1075F80002EB8300D0F8CC447CB1D0F8D04464B11D
:107608004644ABF10B04C0F8C854B379357980F817
:10761800D45480F8D534C0F8C444114B0BF1100B86
:107628005B4523D05BF8075CB1E718463960FBF788
:107638009BF8FB683968C3F8D004D3E72046396063
:10764800FBF792F8FB683968C3F8CC04C5E700BFBC
:10765800F8140020EC11002000540040800900209C
:10766800AB8700088B87000884110020D2F8C43447
:107678001446002B65D0987BD2F8D034D2F8C85481
:10768800D2F8CC649846FFF77BF98A4B9D4200F00C
:107698007182894A136B23F0100313631021864A01
:1076A800136B0B4313631EB115220123B271F371DF
:1076B80094F8D534002B30460CBF1E213E210422FD
:1076C800FBF716F9404630B116220123414688F8E7
:1076D800062088F8073094F8D534002B0CBF1E21FB
:1076E8003E2140460422FBF703F92A6894F8D46443
:1076F800724B734822F001022A602968714A002EF1
:1077080018BF03460A402A602B612A68002342F00A
:1077180001022A60AB60EB60AB60AB6843F40043E6
:10772800AB602B682B606B6823F0784323F400432D
:107738006B602B6823F400332B602B6843F0010344
:107748002B60614B614A5E799D79DAF800E0604B05
:10775800A6F10101B1FA81F149090846A5F1010133
:10776800B1FA81F14909012E10701171CEF3C030C0
:107778004FF000011960907059609960D9601961E3
:107788000EF4004004BF5178197008B1D178D9734C
:10779800917909B1D1799972012D04BF52795A7141
:1077A8004B4B1A4600234FF0070816461D467A61D0
:1077B8003278FB60104600213A61FBF769FD3A69AF
:1077C800FB68834648BB08F101085FFA88F8B8F1FE
:1077D8000B0F06F10506EBD1002B38D0364BDFF83E
:1077E800FCB0DA6A22F4F872DA62DA6A42F4D87221
:1077F800DA623C20FFF7C4F8786936495A46002314
:10780800064603E001330C2B00F0F28150688842F1
:1078180002F11C02F6D17E61ECE11046FAF7A4FFF2
:10782800132120B14FF0000380F80680C371FBF7E5
:1078380031FA3078FBF746FD691C707001224FF071
:107848000700B5705B463071CDB2F270BBE7DFF868
:107858008CB001210846FBF7F9FB00210846FBF72D
:10786800F5FB00210220FBF7F1FB0A25D9F80400FB
:10787800FBF7CCFBD9F80000FBF7C8FBFEF774FF59
:10788800FEF772FF013DF1D129462846FBF7DEFBE2
:1078980029460120FBF7DAFB4FF4197229460E48F6
:1078A80000F041FFFCF7E6F9002846D00A4E4FF0F9
:1078B800CC0818E000580040001002407A25E0008B
:1078C800300E5000FFE0CF00E01500202811002006
:1078D800F015002008000240C009002034000020F4
:1078E800D5B2022D29D808FB05F37B61F3586A1C31
:1078F800002BF5D1C2783B61A24B90F9020003EB53
:107908008202D2F88C10FCF78DF8814605EB450011
:1079180000EB0010B9F1000F0BD03B6906EB8000BB
:107928001946CC2200F0FFFE7B69013546F803902A
:10793800EDB2FCF735F80028D3D1934E934BC4F839
:10794800EC343046FCF7F0FC00250122FF2322200E
:1079580084F8F82484F8FA5484F8F934FAF704FF20
:10796800C4F8FC0410B12623C57183714921FBF7C3
:1079780091F9D4F8FC04864DFBF752FB6420FAF722
:1079880025FCD4F8FC04FBF751FB2C20FAF7ECFE9D
:10799800286018B11D2200238271C371DFF84C8260
:1079A8000D21FBF777F92868FBF740FBB8F80030A2
:1079B80023F040031B041B0CA8F80030B8F8003073
:1079C8009BB223F0380343F01003A8F80030B8F84E
:1079D80000309BB243F04003A8F800300A20FEF7BD
:1079E800EDFF4020FEF7EAFF8A20FEF7E7FFFF20C1
:1079F800FEF7E4FFB8F80030286823F040031B04C2
:107A08001B0CA8F80030B8F800309BB223F03803FC
:107A180043F00803A8F80030B8F800309BB243F0F0
:107A28004003A8F80030FBF7FBFA0020FEF7C6FF7A
:107A38000220FEF7C3FF2868FBF7F8FA554B564AB1
:107A4800597898781B781370C1F12001C0F11000A3
:107A58000023C02284F8001584F801054F4903204B
:107A6800FEF7ECF94848F9F7C7FAD4F8EC344C4A71
:107A78009B681660444898470126FF2384F8F864F9
:107A880084F8F934A0245FFA86F823460025B14625
:107A9800434A1068E9B20E1D0268867280F80B80AE
:107AA8000331966901340135C9B24246B047E4B2A0
:107AB800182D234657D0FF2CEAD13A4A3A4907F104
:107AC8003000FBF795FE364807F1300306221421F3
:107AD8000068FBF7C7FB324A344B10680D210622B9
:107AE800FBF7C0FB2E4B186803685B6A9847DAF807
:107AF80000302F4A01219B02117000F158822D4954
:107B08002D4D2E482E4A2F4C04230B702B7000212C
:107B18002D4B018064205960197058702B4B1180CF
:107B28005B792B4A2170012B1180518000F035823E
:107B3800264B284A997928480023012903701360A5
:107B48005360936000F0AE84244B1B68CAF8003081
:107B5800FFF768FA224B224A1B7863F07F03137001
:107B6800FCF788FCFCE74E460136052EA5D0FF2C15
:107B7800A3D088E71B4A1C49136B23F02003136327
:107B88008DE500BF40870008A8090020A0870008ED
:107B980090160020300C0020941600206D5B000821
:107BA8004C0C0020948B00089C8B0008A08B0008CC
:107BB800500C0020781C0020881C00207C1C002011
:107BC8007A1C0020CC150020801C0020E015002025
:107BD80044160020D0150020791C00202C0C002011
:107BE8002210002000100240200000100038004041
:107BF8007E610023C3EBC3030BEB8303AC4E19690F
:107C08007269AC480A437261002606221A765E76CB
:107C18008046F9F71BFB07F13000F9F7E9FA022D66
:107C280034BF33468023A449A44A7B6439634FF4A4
:107C380080734FF4806140467A63BB6420224FF41E
:107C48000053F96407F130013A65BE633E64BE65CE
:107C58007B65BD87F9F7DAFAD8F800304FF0A0460F
:107C680043F00103C8F80030B36823F04053B36011
:107C7800B36843F08053B360FEF7F0FCB36823F0B9
:107C88008043B360B368B360B36843F00043B36044
:107C98007B691A46B368002BFCDBB0687A6120F078
:107CA8004050B060B0688649864A874B40F0005023
:107CB800B0608868024042F468328A60F268134013
:107CC80043F40053F360326B6B1E22F00F02134330
:107CD80033634FF0A04001234FF007081F2506E04B
:107CE8007A697A49053291427A6100F03B817A6972
:107CF800D278002AF4D079695E1C042B91F801E04F
:107D08000979F6B200F2278403EB43035B00026BA8
:107D180005FA03FC22EA0C020EFA03F31343036389
:107D2800BEF1090F00F204840EF1FF334269426983
:107D380003EB43034FF0380E0EFA03FE22EA0E025D
:107D48004261DA1C436901FA02F21A43426133467E
:107D5800C6E7A94538BF4C4606D2616820461434A8
:107D6800FEF7D6FEAC42F8D3594A5A4CDFF8848164
:107D780001231381BB60584BE31AFB6003233B616B
:107D88000026554B3B63FB68BE63FE633E647E641E
:107D98007B63D8F81030180606D5504BC8F8043065
:107DA80003F18833C8F804303B7A87F84430A520BB
:107DB8003423C8F80C300222BE2307F118013876A4
:107DC80007F130007B76FBF795FA022207F11801DC
:107DD8004FF6FF70FEF7C4FFA945834633D2404BE8
:107DE8007B617A6987F82D60B2F802A01388CAF31C
:107DF8000B0AC3F30B000AF106011B0B0622398597
:107E0800788507F1280107F1300087F82C30FBF757
:107E180071FA5846062207F12801FEF7A1FF7B698F
:107E280083465968524607F13000FBF763FA7B69CD
:107E380058465968524614337B61FEF791FF7B69B7
:107E4800AB428346CDD3022207F11C0107F1300073
:107E5800BE83FBF74FFA022207F11C015846FEF7D2
:107E68007FFF43BADB43022207F1280107F1300004
:107E78003B85FBF73FFAF86B002840F04983386CE4
:107E880097F84430002B40F01F83002840F01683F9
:107E9800FEF77FFF00287FF4EFA90520FDF78CFA95
:107EA8001049114B1148124A0860DA60FFF7E4B92B
:107EB8000010024008000240400000500416002054
:107EC80000030050E010FCFF07C0FFFD041600206F
:107ED800F81400200000040800F003082301674597
:107EE800388C0008FC9F002000ED00E0EFBEADDEFE
:107EF8000400FA05002002409A4A9B4B12211160A7
:107F08005A685A605A685A605A6842F480625A60DD
:107F18005A6822F47C125A605A6842F4E8125A608D
:107F28001A6842F080721A601A689401FCD55A687F
:107F38008D4922F003025A605A6842F002025A60E0
:107F48004B6803F00C03082BFAD1FFF73CB9002269
:107F58001A6062B6854B1B6883F30888844B1B68DC
:107F68009847FEE74FF0A0421346916841F001019F
:107F780091601A68D207FCD5DA6822F00202DA604A
:107F8800DA6842F00202DA60DA6842F00102DA6086
:107F98009A6842F004029A605BE42822754800F06F
:107FA800C2FB9FED750A7548FBF7D4FAC0E5744B20
:107FB800DA7A1B7816463AB1022B00F05E82032B60
:107FC80000F052828B4209D06E4B00221A706E4B21
:107FD8006D4A1B7843F00803137090E56B4C6C48AE
:107FE8006C49237018224FF43473C4F8E4026260B9
:107FF800A16004F114001A460021236100F093FBEC
:108008003046FBF7D7FB6449C36802680A60054637
:10801800002B00F03F813046FAF7A6FB5F4B186053
:1080280018B12A2200238271C3712A7A4E21FAF7E5
:108038005FFC4D4A287C536959491E46C0EBC00372
:108048000BEB830BDBF81030334353614FF0000622
:108058002A2200238BF818208BF81960C022FDF71C
:10806800EDFE4D4B1868FAF76DF8FEF789FCA0880D
:108078004C494D4A484B01FB00F191421B6840F3C3
:10808800E88100218C4649481988A668B2FBF6F2B7
:108098008342C2F34E0EA4F80CE092B289B200F00B
:1080A800D48100F50060834200F0CF81B3F1804FA6
:1080B80000F0CB81A0F59830834200F0C68100F52E
:1080C8008060834200F0C1813948834200F0B88162
:1080D80000F58060834200F0B38121F4407100F51F
:1080E8008C3089B283421980DA62A3F828C000F084
:1080F800A481304A934200F0A08102F54062934285
:1081080000F09B8102F58062934200F0968102F5AF
:108118008062934200F091810121596195F807E04E
:108128001EF0020240F0848193464FF480706A7911
:108138001EF0010F0CBF4FF000084FF002080C2A88
:1081480000F25581DFE812F00E015301530153018B
:10815800E600530153015301B20053015301530187
:10816800380000BF002002400010024000D8FF1F66
:1081780004D8FF1F54160020CDCCCC3D5816002043
:1081880000120020DD1A0020221000200C1200200E
:1081980010880008CE070700EC1A002024100020E1
:1081A800211C000840420F0000A24A04002C014094
:1081B80000100040003401401A6ADFF84CC322F472
:1081C80080521A621A6AD3F804E0DE6922F4005277
:1081D80042EA013226F4E64141F4C041634542EAED
:1081E80008320E4600F08880BB498B4200F084803C
:1081F8000021C3F804E0DE6119641A62DA6942F406
:108208000062DA615A6CE86842F400425A64B34A80
:10821800036810604FF6FE7213400360F9F716F812
:1082280007F13000F8F7E4FFAD4B6A791B68216964
:10823800B98734331344A94A3B631068DFF8CCE2AA
:10824800C7F834E010228023002407F13001BA6314
:108258007B644FF480724FF40053BA647B65BC654D
:108268003C64FC643C65F8F7D1FF6A799C4B0C2AA6
:10827800196898BF9B4BC86896BF03EB4202234618
:10828800B2F8D830954A03431268CB60136843F0BC
:1082980002031360944C01252570FBF77BFA2378C1
:1082A800002B3FF494AE914B1D7090E61A6ADFF8EC
:1082B800589222F480721A621A6AD3F804C0D3F86A
:1082C8001CE022F4007242EA01222EF0730E4B45A4
:1082D80042EA08224EF0600E13D07F498B4210D03C
:1082E8000021C3F804C0C3F81CE0D9631A62DA6934
:1082F80042F00802DA6185E72EF4804E4EEA801ECD
:1083080076E722F440622CF4405C42EA0B224CEA05
:10831800001CE5E71A6ADFF8F09122F010021A62F1
:108328001A6AD3F804C0D3F818E022F020022EF01D
:10833800807E42EA01122EF4E64E4B4542EA0818C6
:108348004EF4C04141D0644A93423ED00020C3F865
:1083580004C099619863C3F820809A6942F4006266
:108368009A614FE71A6ADFF8A09122F001021A62B7
:108378001A6AD3F804C0D3F818E022F002022EF4E7
:10838800803E0A432EF0730E4B4548EA02084EF031
:10839800600123D0504A934220D002F540629342B4
:1083A8001CD002F58062934218D002F58062934295
:1083B80014D00020C3F804C099615863C3F8208022
:1083C8009A6942F008029A611CE728F0C0082CF468
:1083D800406C48EA0B184CEA800CB7E728F00C0808
:1083E8002CF4407C4BEA080840EA0C0CE1E70C2A24
:1083F8003FF608AF01A151F822F000BFC983000879
:108408000D8200080D8200080D82000863830008B1
:108418000D8200080D8200080D820008F78200080E
:108428000D8200080D8200080D82000805820008F0
:10843800002004220146934679E600221A866BE65C
:108448001980DA62A3F828C066E621F0700189B2C3
:108458003AE602EB5100B0FBF1F1013989B28C46E2
:108468000131B2FBF1F20EE6214C224BC4F8E432A2
:108478001222C82349F27041B9E51D4C1E4BC4F8BD
:10848800E4324FF41B75002318214AF29E326160D2
:10849800A26004F1140019462A462370256100F0F1
:1084A80042F9ADE5154A9FED160A16481360536068
:1084B8009360D360FBF74EF8FFF746BB3B69013B7F
:1084C8003B617FF45EACE8E4D8F8103043F08003F9
:1084D800C8F81030D9E400BF00340140E81A002081
:1084E800EC1A002040870008DD1A0020DE1A002060
:1084F8000C120020148800080C88000810160020B0
:10850800CDCCCC3E20160020002C014020120020AB
:1085180007F13803C0F104020021184400F003F900
:10852800B96B07F13000FEF79AFAFE633864A7E4E6
:10853800AEF10A028369836902EB420208FA02FE7D
:1085480023EA0E038361836901FA02F21A43826106
:108558003346FFF7C5BB092B0ED8053B03EB430396
:108568005B00426B05FA03FC22EA0C020EFA03F3E5
:1085780013434363FFF7D4BB0E2B0ED80A3B03EB20
:1085880043035B00826B05FA03FC22EA0C020EFA35
:1085980003F313438363FFF7C3BBA3F10F0202EB9B
:1085A80042025200C36B05FA02FC23EA0C030EFADE
:1085B80002F21343C363FFF7B3BB00BF38B5444BA4
:1085C8001A68107810F07F0004D1537A23F0200342
:1085D800537238BD022878D15388002B76D113798D
:1085E800002B73D1537923F08000840004F180417B
:1085F80001F5B8415DB20968002DB4BF01F0300142
:1086080001F44051032860D800295ED0927A002AEC
:108618005BD004F1804404F5B844002D226824DAC4
:1086280002F03002102A4AD103F07F039A0002F1C7
:10863800804202F5B8421368590608D5136840F617
:108648000F710B4043F4004343F0C00313601368F9
:1086580023F4E04323F040039BB283F0300343F458
:10866800004343F08003136029E002F44052B2F55E
:10867800805F24D128B9174B93F82C10F8F7D8FC51
:1086880010E09B0003F1804303F5B8431A685204D5
:1086980008D51A6840F60F710A4042F4404242F089
:1086A80080021A60236823F4804323F070039BB28E
:1086B80083F4405343F4004343F080032360064BA4
:1086C8001B685B699847002038BD022038BD00BF91
:1086D80078150020840100209C15002010B5431E49
:1086E8000A44914200D110BD11F8014B03F8014F23
:1086F800F7E7884210B501EB020303D8421E9942FE
:108708000CD110BD9842F9D28118D21AD34200D1A7
:1087180010BD13F8014D01F8014DF7E711F8014BB1
:1087280002F8014FEBE702440346934200D1704739
:1087380003F8011BF9E700000000000000380140C1
:1087480000000000000000001A2735001926340038
:108758004E0725505000000002000000004800406D
:1087680000000000000000002B3B00002A3A000037
:10877800720727405000000000000000005400402D
:108788001F26281E27297500000000000000000091
:1087980000000000000000005D3E0008613E000887
:1087A80031430008C9400008513E0008213E000836
:1087B800A50F0008990F0008950F00080110000880
:1087C8008D0F00080000000080250000004B00000D
:1087D8000096000000E1000000C2010000840300D0
:1087E80090D00300801A06000008070020A10700A7
:1087F80000100E0040420F0060E3160080841E0047
:1088080070B02500B91B00081D1B0008691A000874
:10881800000200000000000000040000000000004A
:10882800000800000000000000100000901C00205C
:10883800901D0020FFFF0000000000000010203005
:1088480031310000FFFFFFFFFFFF040000001300AD
:10885800002C01404B1B000000000040601C000081
:1088680000040040611D000000080040621E000076
:108878000010004064000000001400406500000083
:10888800003401404D2E0000004001405018000007
:10889800004401405119000000480140521A0000EC
:1088A8003132333435360000100101110102120152
:1088B8000313010414020115020216020317080427
:1088C80020040C21040122020C2C08032D04052E7F
:1088D80008042F0805300306310307320308330361
:1088E8000934020535020B00080C00080D000C07BE
:1088F800000C08000C09000C0A000C0B00040D0009
:108908000C0600040200040E00040F00041000040A
:108918000300080100080200030A640105000000C2
:108928004D1C0008D5240008311D0008DD1C000876
:10893800FD250008191D00083D250008000000005D
:1089480000000000000000000004004020080400AF
:10895800020000001C00024001000000000400406A
:10896800210C040002000000300002400200000058
:108978000044014024000400010000006C00024093
:108988000500000000480140250004000A0000001E
:108998008000024006000000002C01401800200062
:1089A800060000001C00024001000000000000005A
:1089B80000000000000000000000000000000000AF
:1089C800000000000000000000000000000000009F
:1089D800000000000000000000000000000000008F
:1089E800000000000000000000000000000000007F
:1089F800000000000000000000000000000000006F
:108A0800000000000000000000000000000000005E
:108A1800000000000000000000000000000000004E
:108A2800000000000000000000000000000000003E
:108A380000000000000000009F5300084D6100087E
:108A480089530008696300085F61000859610008DC
:108A58005D6100081D6300088D53000895530008E8
:108A6800140002006E0A010100123456789ABC0004
:108A78000000000001069411102702099411102724
:108A88000301E457881300090408030906070106CF
:108A98000907080206000000A1100008A11000083C
:108AA800C5620008A1100008A1100008A110000864
:108AB800A110000811630008A1100008A110000807
:108AC800A1100008A1100008A1100008A1100008BA
:108AD8001201000202000040830440570002010214
:108AE800030100003203530054004D0033003200EC
:108AF80020005600690072007400750061006C0067
:108B0800200043004F004D00200050006F0072000D
:108B180074002000200000002603530054004D007C
:108B28006900630072006F0065006C0065006300F7
:108B3800740072006F006E0069006300730000002B
:108B4800040309040401000009024300020100C0F3
:108B58003209040000010202010005240010010589
:108B680024010001042402020524060001070582ED
:108B7800030800FF09040100020A000000070503BA
:108B8800024000000705810240000000332E332E0A
:108B980030000000562573004F5344004254464CA1
:108BA8000000000044656320313020323031370046
:108BB80031393A34303A31340000000065393932FD
:108BC800323231383400000057414954494E472069
:108BD800464F52204643000053595354454D000018
:108BE80053455249414C0000424154544552595F43
:108BF800564F4C5441474500424154544552595FE1
:108C080043555252454E5400424154544552595FBF
:108C1800414C4552545300005452414E53504F4E0C
:108C2800444552004F53445F534C415645000000A1
:108C3800130004002C0C0020380C00200000000059
:108C48008C8D000812200800240C00203C0C002009
:108C580000000000908D000802020300300C002084
:108C6800440C002000000000000000000102050084
:108C7800640E00201410002000000000653E00086B
:108C8800FE010900281100201C110020000000002E
:108C9800551A000806020800841100207C110020E3
:108CA80000000000B92600080802090098110020F9
:108CB8008C1100200000000023250008F9010400A1
:108CC800A8110020A41100200000000015250008AC
:108CD800FD011E00CC110020AC1100200000000096
:108CE800FD2400080D001C00F8140020A415002025
:108CF800000000009543000811000C00001200203D
:108D0800C015002000000000814000080001040098
:108D18000C160020401B002000000000988D000861
:108D28000B201000E0150020441B0020000000006C
:108D38009C8D0008020103007C160020541B0020B3
:108D480000000000753E00080C020100C81B00204E
:108D5800C41B002000000000AC8D00082F0011008B
:108D6800E01B0020CC1B002000000000AE8D000896
:108D7800F7010600FC1B0020F41B00200000000087
:048D8800C08D000892
:108D8C00002020000001534F4633000090010000EA
:108D9C002B21231E64010100000001000A0129009F
:108DAC0001000000000000000000000000000000B6
:0A8DBC0000000000000001000000AC
:108DC6000800000000000000010203040102030481
:108DD60006070809010002000400060008000A0050
:108DE6000C00100020004000800000010000000080
:108DF60000000000000002400800024000000000E1
:108E0600000B000001000000000000000000000050
:108E1600000002401C00024000000000040C00009C
:108E260001000000000000000000000000000240F9
:108E36003000024000000000080D000001000000A4
:108E46000000000000000000000002404400024054
:108E5600000000000C0E00000100000000000000F1
:108E66000000000000000240580002400000000020
:108E7600100F0000010000000000000000000000CC
:108E8600000002406C0002400000000014100000C8
:108E96000100000000000000000000000000024089
:108EA60080000240000000001811000001000000D0
:108EB6000000000000000000000402400804024018
:108EC6000000000000380000020000000000000062
:108ED60000000000000402401C04024000000000E4
:108EE600043900000200000000000000000000003D
:108EF600000402403004024000000000083A00006E
:108F06000200000000000000000000000004024013
:108F160044040240000000000C3B00000200000078
:108F26000000000000000000000402405804024057
:108F360000000000103C00000200000000000000DD
:108F460000000000716500087F6300088F6200085A
:108F56008D620008316200080D6200087B6100081E
:108F6600E9610008C56100088B6100080000000087
:108F760040000000A1100008AD620008A110000822
:108F8600A1100008A1100008A1100008A1100008F7
:108F9600A1100008A1620008E0010000FFFF000028
:108FA600E08B0008000000000000000051400008AF
:108FB600A086010004000000000000000000000080
:108FC600000000000000000000000000000000009B
:108FD600000000000000000000000000000000008B
:108FE600000000000000000000000000000000007B
:108FF600000000000000000000000000000000006B
:10900600000000000000000000000000000000005A
:10901600000000000000000000000000000000004A
:10902600000000000000000000000000000000003A
:10903600000000000000000000000000000000002A
:10904600000000000000000000000000000000001A
:10905600000000000000000000000000000000000A
:1090660000000000000000000000000000000000FA
:1090760000000000000000000000000000000000EA
:1090860000000000000000000000000000000000DA
:1090960000000000000000000000000000000000CA
:1090A60000000000E88B0008000000002D1A0008F0
:1090B60089010008102700000600000000000000DB
:1090C600000000000000000000000000000000009A
:1090D600000000000000000000000000000000008A
:1090E600000000000000000000000000000000007A
:1090F600000000000000000000000000000000006A
:10910600000000000000000000000000F08B0008D6
:109116000000000000000000793F0008204E00001B
:109126000300000000000000000000000000000036
:109136000000000000000000000000000000000029
:10914600008C00080000000000000000853E0008BA
:10915600204E000003000000000000000000000098
:1091660000000000000000000000000000000000F9
:1091760000000000108C0008000000000000000045
:10918600FD6D0008400D0300030000000000000014
:1091960000000000000000000000000000000000C9
:1091A6000000000000000000208C00080000000005
:1091B60000000000D1430008A00F000001000000DD
:1091C6000000000000000000000000000000000099
:1091D6000000000000000000000000002C8C0008C9
:1091E60000000000C10F0008610F00081A410000CE
:1091F6000500000000000000000000000000000064
:109206000000000000000000000000000000000058
:10921600010000000000000000000000010203043D
:10922600060708090100000000C20100000008004E
:10923600488B000804000000208B00082600000070
:10924600EC8A000832000000A00400201A0000008A
:10925600508B000843000000D88A00081200000066
:109266001A03530054004D00330032000000000082
:0C927600000000000000000000000000EC
:0400000508000000EF
:00000001FF
